:020000040000FA
:1000000000020400000000003669000042690000A0
:100010004E6900005A6900006669000072690000BC
:100020007E690000966900008A6900008A69000004
:100030008A6900008A6900008A6900008A690000F4
:100040008A690000066B00008A6900008A69000066
:100050008A690000306500008A6900008A69000032
:100060008A6900008A6900008A6900008A690000C4
:100070008A6900008A6900008A6900008A690000B4
:100080008A6900008A6900008A6900008A690000A4
:100090008A6900008A6900008A6900008A69000094
:1000A0008A690000EA6700008A6900008A69000026
:1000B0008A6900008A6900008A6900008A69000074
:1000C0008A6900008A6900008A6900008A69000064
:1000D0008A6900008A6900008A6900008A69000054
:1000E0008A6900008A6900008A6900008A69000044
:1000F0008A6900008A6900008A6900008A69000034
:100100008A6900008A6900008A6900008A69000023
:100110008A6900008A6900008A6900008A69000013
:100120008A6900008A6900008A690000006800008E
:10013000066800008A6900008A6900008A69000078
:100140008A6900008A6900008A6900008A690000E3
:100150008A6900008A6900008A6900008A690000D3
:100160008A6900008A6900008A6900003868000016
:100170000C680000226800008A6900008A6900009B
:100180008A6900008A6900008A6900008A690000A3
:100190008A6900008A6900008A6900008A69000093
:1001A0008A6900008A6900008A6900008A69000083
:1001B0008A6900008A6900008A6900008A69000073
:1001C0008A6900008A6900008A6900008A69000063
:1001D0008A6900008A6900008A6900008A69000053
:1001E0008A6900008A6900008A6900008A69000043
:1001F0008A6900008A6900008A6900008A69000033
:100200008A6900008A6900008A6900008A69000022
:100210008A6900008A6900008A6900008A69000012
:100220008A6900008A6900008A6900008A69000002
:100230008A6900008A6900008A6900008A690000F2
:100240008A6900008A6900008A6900008A690000E2
:100250008A6900008A6900008A6900008A690000D2
:100260008A6900008A690000FFFFFF00FFFFFF00AE
:10027000FFFFFF00FFFFFF00FFFFFF00FFFFFF008A
:10028000FFFFFF00FFFFFF00FFFFFF00FFFFFF007A
:10029000FFFFFF00FFFFFF00FFFFFF00FFFFFF006A
:1002A000FFFFFF00FFFFFF00FFFFFF00FFFFFF005A
:1002B000FFFFFF00FFFFFF00FFFFFF00FFFFFF004A
:1002C000FFFFFF00FFFFFF00FFFFFF00FFFFFF003A
:1002D000FFFFFF00FFFFFF00FFFFFF00FFFFFF002A
:1002E000FFFFFF00FFFFFF00FFFFFF00FFFFFF001A
:1002F000FFFFFF00FFFFFF00FFFFFF00FFFFFF000A
:10030000FFFFFF00FFFFFF00FFFFFF00FFFFFF00F9
:10031000FFFFFF00FFFFFF00FFFFFF00FFFFFF00E9
:10032000FFFFFF00FFFFFF00FFFFFF00FFFFFF00D9
:10033000FFFFFF00FFFFFF00FFFFFF00FFFFFF00C9
:10034000FFFFFF00FFFFFF00FFFFFF00FFFFFF00B9
:10035000FFFFFF00FFFFFF00FFFFFF00FFFFFF00A9
:10036000FFFFFF00FFFFFF00FFFFFF00FFFFFF0099
:10037000FFFFFF00FFFFFF00FFFFFF00FFFFFF0089
:10038000FFFFFF00FFFFFF00FFFFFF00FFFFFF0079
:10039000FFFFFF00FFFFFF00FFFFFF00FFFFFF0069
:1003A000FFFFFF00FFFFFF00FFFFFF00FFFFFF0059
:1003B000FFFFFF00FFFFFF00FFFFFF00FFFFFF0049
:1003C000FFFFFF00FFFFFF00FFFFFF00FFFFFF0039
:1003D000FFFFFF00FFFFFF00FFFFFF00FFFFFF0029
:1003E000FFFFFF00FFFFFF00FFFFFF00FFFFFF0019
:1003F000FFFFFF00FFFFFF00FFFFFF00FFFFFF0009
:100400006FEB2100A0F12100000188000000000036
:10041000EE5B020000000000000020004070880039
:10042000000020005070880000002000307088001C
:1004300000002000607088000000200070708800BC
:10044000000020000070880000002000207088005C
:1004500000002000C070880000002000D0708800DC
:1004600000002000E070880000002000F07088008C
:10047000F00F20008070880000002000A07088002D
:1004800000002000407188000000200050718800AA
:10049000000020006071880000002000707188005A
:1004A000E0012F000071880000002000207188000A
:1004B00000002000C071880000002000D07188007A
:1004C00000032300B071880000002000E071880064
:1004D00000002000F0718800000024008071880076
:1004E00080032300A0718800000020004072880073
:1004F0000000200050728800000020006072880018
:100500000000200070728800200020000072880027
:10051000100820002072880000002000C0728800AF
:1005200000002000D072880000002300B072880014
:1005300000002000E0728800000222008072880023
:1005400000012100A0728800000020004073880094
:1005500000002000507388003000240030738800B1
:100560000000200060738800000020007073880085
:1005700020082000007388001000200020738800ED
:1005800000002000C0738800F0CF2000D0738800E6
:1005900000002000B073880000002000E073880095
:1005A000F0CF20008073880000002000A073880036
:1005B000000020004074880000002700507488006C
:1005C000F00F200030748800000020006074880064
:1005D00000002700007488000000280020748800B4
:1005E00000002000C074880000002000D074880043
:1005F00000002000B074880000002000E074880033
:10060000000022008074880000002C00A074880084
:1006100010032000203688001005200030368800A6
:10062000D0062000B036880010072000C0368800B1
:100630000030200040348800001020006034880022
:1006400000B02100B034880000D02100C034880000
:1006500010302300103A880020002000203A880043
:10066000A0082000303A880075AEA80075CEA8001A
:1006700000802A0000118800004C22001011880020
:10068000701C20004011880000802A008011880022
:10069000004C22009011880060022000C0118800E8
:1006A00060802A008012880000402000901288009C
:1006B000701C2000C012880060802A00801588000D
:1006C000004C200090158800701C2000C015880088
:1006D000158EA80004CEA900A0072100B0838800D1
:1006E000C0838800601A2100108D8800208D88004A
:1006F000A020210030908800409088002014210024
:10070000F0898800008A8800E08D2100D0C688002A
:10071000E0C68800000228008008880050442000BD
:1007200060088800CA38EF00D038EF00F0FF2F00D3
:1007300090C68800A0C688006030EF000230EF004D
:100740006988A90069A8A90069C8A8006888A800E4
:1007500068A8A90068C8A8004388A80043A8A90001
:1007600043C8A8001A5B02000000000065CEA80084
:100770001A5B020000000000000420007C5C020004
:100780000000000000032000FA5B020000000000EF
:1007900070082000FA5B02000000000070002000DA
:1007A000FA5B02000000000070022000FA5B020009
:1007B00000000000F0022000FA5B020000000000D0
:1007C000F00E2000FA5B0200000000008002200012
:1007D000FA5B02000000000000002000FA5B02004B
:1007E00000000000400420007C5C020000000000CB
:1007F00000002000FA5B0200000000000000200062
:10080000FA5B020000000000000F2000FA5B02000B
:100810000000000000082000FA5B02000000000059
:1008200050022000FA5B020000000000000F2000D0
:10083000FA5B02000000000000002000FA5B0200EA
:1008400000000000B0042000FA5B0200000000007D
:1008500000002000FA5B0200000000000000200001
:10086000FA5B020000000000A00520007C5C020092
:100870000000000000002000FA5B02000000000001
:10088000B00520007C5C0200000000001000200089
:10089000FA5B020000000000800520007C5C020082
:1008A0000000000060052000FA5B0200000000006C
:1008B000545D020000000000600420007C5C020027
:1008C0000000000000002000FA5B020000000000B1
:1008D00000002000FA5B020000000000D0052000AC
:1008E0007C5C02000000000040002000FA5B020077
:1008F0000000000070002000FA5B02000000000011
:10090000900520007C5C020000000000C004200074
:100910007C5C020000000000154EA80015EEA90046
:1009200015CEA90015AEA8000000000000000000D0
:1009300000000000000000000000000000000000B7
:1009400000000000152EA800825B020000000000DD
:10095000825B020000000000825B020000000000D9
:10096000825B020000000000C05A0200000000008C
:10097000825B020000000000825B020000000000B9
:10098000825B020000000000825B020000000000A9
:1009900015EEA80015CEA80015AEA80000000000B6
:1009A0000000000000000000000000000000000047
:1009B0000000000000000000152EA800825B02006D
:1009C00000000000825B020000000000825B020069
:1009D00000000000825B020000000000C05A02001C
:1009E00000000000825B020000000000825B020049
:1009F00000000000825B020000000000825B020039
:100A00000000000015EEA90015CEA90015AEA90042
:100A100000000000000000000000000000000000D6
:100A2000000000000000000000000000152EA800DB
:100A3000825B020000000000825B020000000000F8
:100A4000825B020000000000825B020000000000E8
:100A5000C05A020000000000825B0200000000009B
:100A6000825B020000000000825B020000000000C8
:100A7000825B020000000000156EA900000000006B
:100A80000000000000000000000000000000000066
:100A90000000000000000000800E2000E25902006B
:100AA0000000000000002000E259020000000000E9
:100AB00000002000E25902000000000000002000B9
:100AC000E25902000000000000002000E25902008C
:100AD0000000000000002000E259020000000000B9
:100AE00000002000E2590200000000000000200089
:100AF000E259020000000000365A02000000000027
:100B000000027800365A0200000000004800DD00B4
:100B100004004000F0808800365A02000000000007
:100B200000027800365A0200000000004800DD0094
:100B30000400400000818800365A020000000000D6
:100B400000027800365A0200000000004800DD0074
:100B50000400400010838800365A020000000000A4
:100B600000027800365A0200000000004800DD0054
:100B70000400400020838800365A02000000000074
:100B800000027800365A0200000000004800DD0034
:100B90000400400030838800365A02000000000044
:100BA00000027800365A0200000000004800DD0014
:100BB0000400400040838800365A02000000000014
:100BC00000027800365A0200000000004800DD00F4
:100BD0000400400050838800365A020000000000E4
:100BE00000027800365A0200000000004800DD00D4
:100BF0000400400001052000810050004220AF00A9
:100C000010060400000000003104200081005000A4
:100C10004220AF0010060400000000000005200084
:100C200060838800365A020000000000000278004D
:100C3000365A0200000000004800DD0004004000B9
:100C400070838800365A020000000000000278001D
:100C5000365A0200000000004800DD000400400099
:100C6000E0808800365A0200000000000002780090
:100C7000365A0200000000004800DD000400400079
:100C8000F0938800365A020000000000000278004D
:100C9000365A0200000000004800DD000400400059
:100CA00000948800156EA8000000000000000000FD
:100CB0000000000000000000000000000000000034
:100CC0000000000015EEA80015CEA80015AEA80083
:100CD0000000000000000000000000000000000014
:100CE000000000000000000000000000156EA900D8
:100CF00000000000000000000000000000000000F4
:100D0000000000000000000000000000800E200035
:100D1000E25902000000000000002000E259020039
:100D20000000000000002000E25902000000000066
:100D300000002000E2590200000000000000200036
:100D4000E25902000000000000002000E259020009
:100D50000000000000002000E25902000000000036
:100D600000002000E259020000000000365A020094
:100D70000000000000027800365A02000000000067
:100D80004800DD000400400010948800365A02003C
:100D90000000000000027800365A02000000000047
:100DA0004800DD000400400020948800156EA80073
:100DB0000000000000000000000000000000000033
:100DC000000000000000000000000000A628210034
:100DD00010002000005B780050032000005B7800CA
:100DE00010838000001B7800A0002000001B78000A
:100DF00000002000001B7800000A2000001B780083
:100E0000C629210000002000001B780000402600B9
:100E1000001B7800C62B210010002000005B78002A
:100E200050032000005B780010838000001B7800D6
:100E3000A0002000001B780000002000001B7800AC
:100E4000000F2000001B7800E62C2100000020008D
:100E5000001B780000402600001B7800E62E2100D1
:100E600010002000005B780050032000005B780039
:100E700010838000001B7800A0002000001B780079
:100E800000002000001B780000142000001B7800E8
:100E90000630210000002000001B780000402600E2
:100EA000001B78000632210010002000005B780053
:100EB00050032000005B780010838000001B780046
:100EC000A0002000001B780000002000001B78001C
:100ED00000192000001B78002633210000002000AC
:100EE000001B780000402600001B780026352100FA
:100EF00010002000005B780050032000005B7800A9
:100F000010838000001B7800A0002000001B7800E8
:100F100000002000001B7800001E2000001B78004D
:100F20004636210000002000001B7800004026000B
:100F3000001B78004638210010002000005B78007C
:100F400050032000005B780010838000001B7800B5
:100F5000A0002000001B780000002000001B78008B
:100F600000232000001B78006639210000002000CB
:100F7000001B780000402600001B7800663B210023
:100F800010002000005B780050032000005B780018
:100F900010838000001B7800A0002000001B780058
:100FA00000002000001B780000282000001B7800B3
:100FB000863C210000002000001B78000040260035
:100FC000001B7800863E210010002000005B7800A6
:100FD00050032000005B780010838000001B780025
:100FE000A0002000001B780000002000001B7800FB
:100FF000002D2000001B7800A63F210000002000EB
:10100000001B780000402600001B7800A64121004C
:1010100010002000005B780050032000005B780087
:1010200010838000001B7800A0002000001B7800C7
:1010300000002000001B7800A00A2000001B7800A0
:10104000C642210000002000001B7800004026005E
:10105000001B7800C644210010002000005B7800CF
:1010600050032000005B780010838000001B780094
:10107000A0002000001B780000002000001B78006A
:10108000A00F2000001B7800E64521000000200092
:10109000001B780000402600001B7800E647210076
:1010A00010002000005B780050032000005B7800F7
:1010B00010838000001B7800A0002000001B780037
:1010C00000002000001B7800A0142000001B780006
:1010D0000649210000002000001B78000040260087
:1010E000001B7800064B210010002000005B7800F8
:1010F00050032000005B780010838000001B780004
:10110000A0002000001B780000002000001B7800D9
:10111000A0192000001B7800264C210000002000B0
:10112000001B780000402600001B7800264E21009E
:1011300010002000005B780050032000005B780066
:1011400010838000001B7800A0002000001B7800A6
:1011500000002000001B7800A01E2000001B78006B
:10116000464F210000002000001B780000402600B0
:10117000001B78004651210010002000005B780021
:1011800050032000005B780010838000001B780073
:10119000A0002000001B780000002000001B780049
:1011A000A0232000001B78006652210000002000D0
:1011B000001B780000402600001B780066542100C8
:1011C00010002000005B780050032000005B7800D6
:1011D00010838000001B7800A0002000001B780016
:1011E00000002000001B7800A0282000001B7800D1
:1011F0008655210000002000001B780000402600DA
:10120000001B78008657210010002000005B78004A
:1012100050032000005B780010838000001B7800E2
:10122000A0002000001B780000002000001B7800B8
:10123000A02D2000001B7800A658210000002000EF
:10124000001B780000402600001B7800A65A2100F1
:1012500010002000005B780050032000005B780045
:1012600010838000001B7800A0002000001B780085
:1012700000002000001B7800400B2000001B7800BD
:10128000C65B210000002000001B78000040260003
:10129000001B7800C65D210010002000005B780074
:1012A00050032000005B780010838000001B780052
:1012B000A0002000001B780000002000001B780028
:1012C00040102000001B7800E65E21000000200096
:1012D000001B780000402600001B7800E66021001B
:1012E00010002000005B780050032000005B7800B5
:1012F00010838000001B7800A0002000001B7800F5
:1013000000002000001B780040152000001B780022
:101310000662210000002000001B7800004026002B
:10132000001B78000664210010002000005B78009C
:1013300050032000005B780010838000001B7800C1
:10134000A0002000001B780000002000001B780097
:10135000401A2000001B78002665210000002000B4
:10136000001B780000402600001B78002667210043
:1013700010002000005B780050032000005B780024
:1013800010838000001B7800A0002000001B780064
:1013900000002000001B7800401F2000001B780088
:1013A0004668210000002000001B78000040260055
:1013B000001B7800466A210010002000005B7800C6
:1013C00050032000005B780010838000001B780031
:1013D000A0002000001B780000002000001B780007
:1013E00040242000001B7800666B210000002000D4
:1013F000001B780000402600001B7800666D21006D
:1014000010002000005B780050032000005B780093
:1014100010838000001B7800A0002000001B7800D3
:1014200000002000001B780040292000001B7800ED
:10143000866E210000002000001B7800004026007E
:10144000001B78008670210010002000005B7800EF
:1014500050032000005B780010838000001B7800A0
:10146000A0002000001B780000002000001B780076
:10147000402E2000001B7800A671210000002000F3
:10148000001B780000402600001B7800A673210096
:1014900010002000005B780050032000005B780003
:1014A00010838000001B7800A0002000001B780043
:1014B00000002000001B7800E00B2000001B7800DB
:1014C000C674210000002000001B780000402600A8
:1014D000001B7800C676210010002000005B780019
:1014E00050032000005B780010838000001B780010
:1014F000A0002000001B780000002000001B7800E6
:10150000E0102000001B7800E6772100000020009A
:10151000001B780000402600001B7800E6792100BF
:1015200010002000005B780050032000005B780072
:1015300010838000001B7800A0002000001B7800B2
:1015400000002000001B7800E0152000001B780040
:10155000067B210000002000001B780000402600D0
:10156000001B7800067D210010002000005B780041
:1015700050032000005B780010838000001B78007F
:10158000A0002000001B780000002000001B780055
:10159000E01A2000001B7800267E210000002000B9
:1015A000001B780000402600001B780026802100E8
:1015B00010002000005B780050032000005B7800E2
:1015C00010838000001B7800A0002000001B780022
:1015D00000002000001B7800E01F2000001B7800A6
:1015E0004681210000002000001B780000402600FA
:1015F000001B78004683210010002000005B78006B
:1016000050032000005B780010838000001B7800EE
:10161000A0002000001B780000002000001B7800C4
:10162000E0242000001B78006684210000002000D8
:10163000001B780000402600001B78006686210011
:1016400010002000005B780050032000005B780051
:1016500010838000001B7800A0002000001B780091
:1016600000002000001B7800E0292000001B78000B
:101670008687210000002000001B78000040260023
:10168000001B78008689210010002000005B780094
:1016900050032000005B780010838000001B78005E
:1016A000A0002000001B780000002000001B780034
:1016B000E02E2000001B7800A68A210000002000F8
:1016C000001B780000402600001B7800AE6202007C
:1016D00000000000F00F200050938800803E2000A2
:1016E00090838800000020001081880020818800FD
:1016F00000002000709388002828A8002848A8002F
:101700002A28A8002168A8002A48A80020E8A800E4
:10171000C228A80000002000C0C688000230AE0029
:1017200018120400000000000230A900B0072000D9
:10173000E06A02000000000080B02E00E06A0200B3
:101740000000000010838000E06A0200000000003A
:1017500020838000E06A02000000000030838000E7
:10176000E06A02000000000040838000E06A02009E
:101770000000000050838000E06A020000000000CA
:1017800060838000E06A0200000000007083800037
:10179000E06A020000000000F0808000E06A0200C1
:1017A0000000000000818000E06A020000000000EC
:1017B000E0808000E06A020000000000808380007A
:1017C000E06A020000000000F0828000E06A02008F
:1017D00000000000A628210016027800F10F20006A
:1017E000010262004101200006834000964178001A
:1017F00001F02F008181610004807100E06A020025
:1018000000000000A6282100200220000003430061
:1018100016007800E06A020000000000C62B2100DC
:1018200016027800F10F2000010262004101200041
:10183000068340009641780001F02F00818161000D
:1018400004807100E06A020000000000C62B210045
:10185000200220000003430016007800E06A020026
:1018600000000000E62E210016027800F10F200093
:101870000102620041012000068340009641780089
:1018800001F02F008181610004807100E06A020094
:1018900000000000E62E210020022000000343008B
:1018A00016007800E06A0200000000000632210005
:1018B00016027800F10F20000102620041012000B1
:1018C000068340009641780001F02F00818161007D
:1018D00004807100E06A020000000000063221006E
:1018E000200220000003430016007800E06A020096
:1018F000000000002635210016027800F10F2000BC
:1019000001026200410120000683400096417800F8
:1019100001F02F008181610004807100E06A020003
:1019200000000000263521002002200000034300B3
:1019300016007800E06A020000000000463821002E
:1019400016027800F10F2000010262004101200020
:10195000068340009641780001F02F0081816100EC
:1019600004807100E06A0200000000004638210097
:10197000200220000003430016007800E06A020005
:1019800000000000663B210016027800F10F2000E5
:101990000102620041012000068340009641780068
:1019A00001F02F008181610004807100E06A020073
:1019B00000000000663B21002002200000034300DD
:1019C00016007800E06A020000000000863E210058
:1019D00016027800F10F2000010262004101200090
:1019E000068340009641780001F02F00818161005C
:1019F00004807100E06A020000000000863E2100C1
:101A0000200220000003430016007800E06A020074
:101A100000000000A641210016027800F10F20000E
:101A200001026200410120000683400096417800D7
:101A300001F02F008181610004807100E06A0200E2
:101A400000000000A6412100200220000003430006
:101A500016007800E06A020000000000C644210081
:101A600016027800F10F20000102620041012000FF
:101A7000068340009641780001F02F0081816100CB
:101A800004807100E06A020000000000C6442100EA
:101A9000200220000003430016007800E06A0200E4
:101AA00000000000E647210016027800F10F200038
:101AB0000102620041012000068340009641780047
:101AC00001F02F008181610004807100E06A020052
:101AD00000000000E6472100200220000003430030
:101AE00016007800E06A020000000000064B2100AA
:101AF00016027800F10F200001026200410120006F
:101B0000068340009641780001F02F00818161003A
:101B100004807100E06A020000000000064B210012
:101B2000200220000003430016007800E06A020053
:101B300000000000264E210016027800F10F200060
:101B400001026200410120000683400096417800B6
:101B500001F02F008181610004807100E06A0200C1
:101B600000000000264E2100200220000003430058
:101B700016007800E06A02000000000046512100D3
:101B800016027800F10F20000102620041012000DE
:101B9000068340009641780001F02F0081816100AA
:101BA00004807100E06A020000000000465121003C
:101BB000200220000003430016007800E06A0200C3
:101BC000000000006654210016027800F10F20008A
:101BD0000102620041012000068340009641780026
:101BE00001F02F008181610004807100E06A020031
:101BF0000000000066542100200220000003430082
:101C000016007800E06A02000000000086572100FC
:101C100016027800F10F200001026200410120004D
:101C2000068340009641780001F02F008181610019
:101C300004807100E06A0200000000008657210065
:101C4000200220000003430016007800E06A020032
:101C500000000000A65A210016027800F10F2000B3
:101C60000102620041012000068340009641780095
:101C700001F02F008181610004807100E06A0200A0
:101C800000000000A65A21002002200000034300AB
:101C900016007800E06A020000000000C65D210026
:101CA00016027800F10F20000102620041012000BD
:101CB000068340009641780001F02F008181610089
:101CC00004807100E06A020000000000C65D21008F
:101CD000200220000003430016007800E06A0200A2
:101CE00000000000E660210016027800F10F2000DD
:101CF0000102620041012000068340009641780005
:101D000001F02F008181610004807100E06A02000F
:101D100000000000E66021002002200000034300D4
:101D200016007800E06A020000000000066421004E
:101D300016027800F10F200001026200410120002C
:101D4000068340009641780001F02F0081816100F8
:101D500004807100E06A02000000000006642100B7
:101D6000200220000003430016007800E06A020011
:101D7000000000002667210016027800F10F200005
:101D80000102620041012000068340009641780074
:101D900001F02F008181610004807100E06A02007F
:101DA00000000000266721002002200000034300FD
:101DB00016007800E06A020000000000466A210078
:101DC00016027800F10F200001026200410120009C
:101DD000068340009641780001F02F008181610068
:101DE00004807100E06A020000000000466A2100E1
:101DF000200220000003430016007800E06A020081
:101E000000000000666D210016027800F10F20002E
:101E100001026200410120000683400096417800E3
:101E200001F02F008181610004807100E06A0200EE
:101E300000000000666D2100200220000003430026
:101E400016007800E06A02000000000086702100A1
:101E500016027800F10F200001026200410120000B
:101E6000068340009641780001F02F0081816100D7
:101E700004807100E06A020000000000867021000A
:101E8000200220000003430016007800E06A0200F0
:101E900000000000A673210016027800F10F200058
:101EA0000102620041012000068340009641780053
:101EB00001F02F008181610004807100E06A02005E
:101EC00000000000A6732100200220000003430050
:101ED00016007800E06A020000000000C6762100CB
:101EE00016027800F10F200001026200410120007B
:101EF000068340009641780001F02F008181610047
:101F000004807100E06A020000000000C676210033
:101F1000200220000003430016007800E06A02005F
:101F200000000000E679210016027800F10F200081
:101F300001026200410120000683400096417800C2
:101F400001F02F008181610004807100E06A0200CD
:101F500000000000E6792100200220000003430079
:101F600016007800E06A020000000000067D2100F3
:101F700016027800F10F20000102620041012000EA
:101F8000068340009641780001F02F0081816100B6
:101F900004807100E06A020000000000067D21005C
:101FA000200220000003430016007800E06A0200CF
:101FB000000000002680210016027800F10F2000AA
:101FC0000102620041012000068340009641780032
:101FD00001F02F008181610004807100E06A02003D
:101FE00000000000268021002002200000034300A2
:101FF00016007800E06A020000000000468321001D
:1020000016027800F10F2000010262004101200059
:10201000068340009641780001F02F008181610025
:1020200004807100E06A0200000000004683210085
:10203000200220000003430016007800E06A02003E
:10204000000000006686210016027800F10F2000D3
:1020500001026200410120000683400096417800A1
:1020600001F02F008181610004807100E06A0200AC
:1020700000000000668621002002200000034300CB
:1020800016007800E06A0200000000008689210046
:1020900016027800F10F20000102620041012000C9
:1020A000068340009641780001F02F008181610095
:1020B00004807100E06A02000000000086892100AF
:1020C000200220000003430016007800E06A0200AE
:1020D0000000000020808000E06A02000000000094
:1020E00030808000E06A0200000000004080800034
:1020F000E06A02000000000050808000E06A0200F8
:102100000000000060808000E06A02000000000023
:1021100070808000E06A0200000000008080800083
:10212000E06A02000000000090808000E06A020087
:1021300000000000A0808000E06A020000000000B3
:10214000B0808000E06A020000000000C0808000D3
:10215000E06A020000000000D0808000E06A020017
:1021600000000000D0072000E06A0200000000002C
:1021700000402000C1C68000808050004200AE00B8
:102180001812040000000000F093800030948800D2
:10219000009480004094880010948000F0938800A0
:1021A000209480000094880015EEA90015CEA900A7
:1021B00015AEA800000000000000000000000000B4
:1021C000000000000000000000000000000000000F
:1021D0009672020000000000156EA90000000000C9
:1021E00000000000000000000000000000000000EF
:1021F000000000000000000040082000E25902003A
:102200000000000004948000F30720000300620037
:10221000E259020000000000F49380004822DE0032
:1022200003006200E259020000000000F493800005
:10223000F30F200003006200E259020000000000DA
:1022400006202000F46A020000000000000278006E
:102250004800DE00F30F200003006000E259020096
:102260000000000003006200E259020000000000CC
:102270000603E9000600E0004220AE00221104003F
:10228000000000000000000000000000000000004E
:10229000156EA80000000000000000000000000013
:1022A000000000000000000000000000000000002E
:1022B000825B020000000000F272020000000000D9
:1022C0000040200001002000F29380000394800071
:1022D0000200400083804800109488002194880008
:1022E00000002000F0938800000020000094880087
:1022F00015EEA80015CEA80015AEA800000000003D
:1023000000000000000000000000000000000000CD
:1023100000000000000000009672020000000000B3
:10232000156EA90000000000000000000000000081
:10233000000000000000000000000000000000009D
:1023400040082000E25902000000000000002000C8
:10235000E25902000000000000002000E2590200E3
:102360000000000000002000E25902000000000010
:102370001094800000027800F30F2000030060003A
:10238000E2590200000000004822DE000300620063
:10239000E259020000000000209480000002780052
:1023A000F30F200003006000E2590200000000006B
:1023B0004822DE0003006200E25902000000000033
:1023C000156EA800000000000000000000000000E2
:1023D00000000000000000000000000000000000FD
:1023E000825B020000000000F272020000000000A8
:1023F00015EEA90015CEA90015AEA9000000000039
:1024000000000000000000000000000000000000CC
:10241000000000000000000030948000F09388006D
:10242000409480000094880000402000D838B50017
:10243000108180000000D000E10720000100600052
:1024400000060100681404000000000016170400D4
:10245000000000002017040000000000181B04000A
:10246000000000009C48040000000000204B040015
:1024700000000000A6130400000000004C1404003B
:102480000000000080210400000000001627040066
:10249000000000004A4D040000000000AA4D0400A6
:1024A00000000000F6400400000000001244040098
:1024B00000000000C627040000000000E22804001D
:1024C00000000000B62E040000000000D634040016
:1024D00000000000162A040000000000322B040057
:1024E00000000000662C040000000000822D0400A3
:1024F000000000007A350400000000009636040059
:1025000000000000CA37040000000000E6380400A4
:10251000000000001A3A040000000000363B0400EE
:10252000000000006A3C040000000000863D04003A
:1025300000000000A63E040000000000C23F0400AE
:10254000000000004A44040000000000664504004A
:10255000000000009A460400000000005E480400ED
:10256000000000009E130400000000009E13040001
:10257000000000009E130400000000009E130400F1
:10258000000000009E130400000000009E130400E1
:10259000000000009E130400000000009E130400D1
:1025A000000000009E130400000000009E130400C1
:1025B000000000009E130400000000009E130400B1
:1025C000000000009E130400000000009E130400A1
:1025D000000000009E130400000000009E13040091
:1025E000000000009E130400000000009E13040081
:1025F000000000009E130400000000009E13040071
:10260000000000009E130400000000009E13040060
:10261000000000009E130400000000009E13040050
:10262000000000009E130400000000009E13040040
:10263000000000009E130400000000009E13040030
:10264000000000009E130400000000009E13040020
:10265000000000009E130400000000009E13040010
:10266000000000009E130400000000009E13040000
:10267000000000009E130400000000009E130400F0
:10268000000000009E130400000000009E130400E0
:10269000000000009E130400000000009E130400D0
:1026A000000000009E130400000000009E130400C0
:1026B000000000009E130400000000009E130400B0
:1026C000000000009E130400000000009E130400A0
:1026D000000000009E130400000000009E13040090
:1026E000000000009E130400000000009E13040080
:1026F000000000009E130400000000009E13040070
:10270000000000009E130400000000009E1304005F
:10271000000000009E130400000000009E1304004F
:10272000000000009E130400000000009E1304003F
:10273000000000009E1304000000000000002000C4
:10274000108188008E0B040000000000545D020020
:1027500000000000E4112000600420007C5C020006
:1027600000000000F30F200003006200FA5B02008B
:10277000000000004822DE0003006200FA5B020055
:1027800000000000200420007C5C0200000000002B
:1027900030052000FA5B020000000000000220006B
:1027A000FA5B02000000000040052000FA5B020016
:1027B0000000000000022000FA5B020000000000A0
:1027C00050052000FA5B020000000000000220001B
:1027D000FA5B02000000000020042000FA5B020007
:1027E0000000000084482000600420007C5C02009F
:1027F00000000000F30F200003006200FA5B0200FB
:10280000000000004822DE0003006200FA5B0200C4
:1028100000000000200420007C5C0200000000009A
:10282000D0042000FA5B0200000000001004200029
:10283000FA5B02000000000090042000FA5B020036
:1028400000000000E0042000FA5B0200000000002D
:1028500000022000FA5B020000000000D00420000B
:10286000FA5B02000000000050042000FA5B020046
:1028700000000000E0042000FA5B020000000000FD
:1028800050052000FA5B0200000000002230EC003E
:102890008E0B040000000000A0C680003100200064
:1028A000010050004220AE0064140400000000004B
:1028B000722102000000000020002000108188002A
:1028C0008E0B0400000000008E0B040000000000CE
:1028D000545D020000000000641720006004200026
:1028E0007C5C020000000000F30F20000300620087
:1028F000FA5B0200000000004822DE0003006200D4
:10290000FA5B020000000000200420007C5C020052
:102910000000000010042000FA5B0200000000002C
:1029200000022000FA5B020000000000700420009A
:10293000FA5B02000000000000022000FA5B0200C7
:102940000000000020052000FA5B020000000000EB
:1029500000022000FA5B020000000000900420004A
:10296000FA5B02000000000000022000FA5B020097
:102970000000000070042000FA5B0200000000006C
:1029800000022000FA5B020000000000500420005A
:10299000FA5B02000000000000022000FA5B020067
:1029A00000000000C0042000FA5B020000000000EC
:1029B00044212000600420007C5C02000000000034
:1029C000F30F200003006200FA5B02000000000029
:1029D0004822DE0003006200FA5B020000000000F3
:1029E000200420007C5C020000000000C0042000E5
:1029F000FA5B02000000000090042000FA5B020075
:102A00000000000010052000FA5B0200000000003A
:102A100050052000FA5B0200000000009004200036
:102A2000FA5B02000000000040042000FA5B020094
:102A30000000000000022000FA5B0200000000001D
:102A400060042000FA5B0200000000005004200037
:102A5000FA5B02000000000020052000FA5B020083
:102A60000000000040052000FA5B020000000000AA
:102A700090042000FA5B020000000000C004200067
:102A8000FA5B02000000000090042000FA5B0200E4
:102A900000000000A0052000FA5B0200000000001A
:102AA00050042000FA5B0200000000002005200016
:102AB000FA5B0200000000004426200060042000B1
:102AC0007C5C020000000000F30F200003006200A5
:102AD000FA5B0200000000004822DE0003006200F2
:102AE000FA5B020000000000200420007C5C020071
:102AF0000000000010042000FA5B0200000000004B
:102B000000052000FA5B0200000000000005200024
:102B1000FA5B020000000000C0042000FA5B020023
:102B20000000000090042000FA5B0200000000009A
:102B300030042000FA5B02000000000010042000B6
:102B4000FA5B02000000000040052000FA5B020072
:102B50000000000090042000FA5B0200000000006A
:102B6000F0042000FA5B020000000000E0042000F6
:102B7000FA5B02000000000000022000FA5B020085
:102B80000000000000022000FA5B020000000000CC
:102B900050052000FA5B020000000000E004200065
:102BA000FA5B02000000000090042000FA5B0200C3
:102BB0000000000040052000FA5B02000000000059
:102BC000C42D2000600420007C5C02000000000096
:102BD000F30F200003006200FA5B02000000000017
:102BE0004822DE0003006200FA5B020000000000E1
:102BF000200420007C5C0200000000007007200020
:102C0000FA5B02000000000070072000FA5B02007F
:102C10000000000070072000FA5B020000000000C6
:102C2000E0022000FA5B0200000000001006200015
:102C3000FA5B02000000000070062000FA5B020050
:102C40000000000020072000FA5B020000000000E6
:102C500090062000FA5B02000000000070062000D1
:102C6000FA5B02000000000050062000FA5B020040
:102C700000000000C0062000FA5B02000000000017
:102C8000E0022000FA5B0200000000003006200095
:102C9000FA5B020000000000F0062000FA5B020070
:102CA00000000000E0022000FA5B020000000000CB
:102CB000A0072000FA5B02000000000010062000C0
:102CC000FA5B0200000000003435200060042000A0
:102CD0007C5C020000000000F30F20000300620093
:102CE000FA5B0200000000004822DE0003006200E0
:102CF000FA5B020000000000200420007C5C02005F
:102D00000000000060052000FA5B020000000000E7
:102D100050062000FA5B020000000000200720009F
:102D2000FA5B02000000000030072000FA5B02009E
:102D30000000000090062000FA5B02000000000086
:102D4000F0062000FA5B020000000000E006200010
:102D5000FA5B020000000000A0032000FA5B020002
:102D60000000000000022000FA5B020000000000EA
:102D700050042000FA5B0200000000002004200044
:102D8000FA5B02000000000020032000FA5B020052
:102D90000000000000032000FA5B020000000000B9
:102DA00000022000FA5B0200000000001004200076
:102DB000FA5B020000000000C0062000FA5B02007F
:102DC0000000000000072000FA5B02000000000085
:102DD00080062000FA5B02000000000010062000C0
:102DE000FA5B020000000000C435200060042000EF
:102DF0007C5C020000000000F30F20000300620072
:102E0000FA5B0200000000004822DE0003006200BE
:102E1000FA5B02000000000080BB2000E082880016
:102E20002230EC008E0B0400000000005C10E20079
:102E30004220AF002230EC008E0B040000000000A6
:102E4000545D020000000000E41120006004200036
:102E50007C5C020000000000F30F20000300620011
:102E6000FA5B0200000000004822DE00030062005E
:102E7000FA5B020000000000200420007C5C0200DD
:102E800000000000D0042000FA5B020000000000F7
:102E900000022000FA5B0200000000001004200085
:102EA000FA5B02000000000000022000FA5B020052
:102EB0000000000090042000FA5B02000000000007
:102EC00000022000FA5B020000000000E004200085
:102ED000FA5B02000000000000022000FA5B020022
:102EE0000000000000022000FA5B02000000000069
:102EF00000022000FA5B020000000000D004200065
:102F0000FA5B02000000000000022000FA5B0200F1
:102F10000000000050042000FA5B020000000000E6
:102F200000022000FA5B020000000000E004200024
:102F3000FA5B02000000000000022000FA5B0200C1
:102F40000000000050052000FA5B020000000000B5
:102F500064142000600420007C5C0200000000007B
:102F6000F30F200003006200FA5B02000000000083
:102F70004822DE0003006200FA5B0200000000004D
:102F8000200420007C5C020000000000D002200031
:102F9000FA5B020000000000D0022000FA5B020091
:102FA00000000000D0022000FA5B020000000000D8
:102FB000D0022000FA5B020000000000D0022000D6
:102FC000FA5B020000000000D0022000FA5B020061
:102FD00000000000D0022000FA5B020000000000A8
:102FE000D0022000FA5B020000000000D0022000A6
:102FF000FA5B020000000000D0022000FA5B020031
:1030000000000000D0022000FA5B02000000000077
:10301000D0022000FA5B020000000000D002200075
:10302000FA5B020000000000D0022000FA5B020000
:1030300000000000D0022000FA5B02000000000047
:10304000D0022000FA5B020000000000D002200045
:10305000FA5B02000000000004232000600420004E
:103060007C5C020000000000F30F200003006200FF
:10307000FA5B0200000000004822DE00030062004C
:10308000FA5B020000000000200420007C5C0200CB
:103090000000000040042000FA5B02000000000075
:1030A00010042000FA5B0200000000004005200030
:1030B000FA5B02000000000010042000FA5B02002E
:1030C0000000000084252000600420007C5C0200D9
:1030D00000000000F30F200003006200FA5B020012
:1030E000000000004822DE0003006200FA5B0200DC
:1030F00000000000200420007C5C020000000000B2
:10310000D0042000FA5B0200000000001004200040
:10311000FA5B020000000000E0042000FA5B0200FD
:103120000000000010042000FA5B02000000000014
:1031300070042000FA5B0200000000005004200030
:10314000FA5B020000000000D0042000FA5B0200DD
:103150000000000050042000FA5B020000000000A4
:10316000E0042000FA5B020000000000400520009F
:10317000FA5B020000000000843E20006004200092
:103180007C5C020000000000F30F200003006200DE
:10319000FA5B0200000000004822DE00030062002B
:1031A000FA5B020000000000200420007C5C0200AA
:1031B0000000000030052000FA5B02000000000063
:1031C00050042000FA5B02000000000040052000CF
:1031D000FA5B02000000000040052000FA5B0200DC
:1031E0000000000090042000FA5B020000000000D4
:1031F000E0042000FA5B02000000000070042000E0
:10320000FA5B02000000000030052000FA5B0200BB
:103210000000000074092000600420007C5C0200B3
:1032200000000000F30F200003006200FA5B0200C0
:10323000000000004822DE0003006200FA5B02008A
:1032400000000000200420007C5C02000000000060
:1032500000052000FA5B020000000000C00420000E
:10326000FA5B02000000000010042000FA5B02007C
:1032700000000000E0042000FA5B020000000000F3
:1032800040052000FA5B02000000000090042000CE
:10329000FA5B020000000000D0042000FA5B02008C
:1032A0000000000070042000FA5B02000000000033
:1032B000F40B2000600420007C5C02000000000091
:1032C000F30F200003006200FA5B02000000000020
:1032D0004822DE0003006200FA5B020000000000EA
:1032E000200420007C5C020000000000300520006B
:1032F000FA5B02000000000050042000FA5B0200AC
:103300000000000040052000FA5B02000000000001
:1033100040052000FA5B020000000000900420003D
:10332000FA5B020000000000E0042000FA5B0200EB
:103330000000000070042000FA5B020000000000A2
:1033400030052000FA5B0200000000000425200088
:10335000600420007C5C020000000000F30F2000ED
:1033600003006200FA5B0200000000004822DE0059
:1033700003006200FA5B020000000000200420004D
:103380007C5C02000000000070052000FA5B020077
:1033900000000000F0042000FA5B020000000000C2
:1033A00020052000FA5B020000000000B0042000AD
:1033B000FA5B02000000000090042000FA5B0200AB
:1033C00000000000E0042000FA5B020000000000A2
:1033D00070042000FA5B020000000000B427200007
:1033E000600420007C5C020000000000F30F20005D
:1033F00003006200FA5B0200000000004822DE00C9
:1034000003006200FA5B02000000000020042000BC
:103410007C5C020000000000D0042000FA5B020087
:1034200000000000F0042000FA5B02000000000031
:1034300040042000FA5B020000000000500420005D
:10344000FA5B0200000000004440200060042000FD
:103450007C5C020000000000F30F2000030062000B
:10346000FA5B0200000000004822DE000300620058
:10347000FA5B020000000000200420007C5C0200D7
:103480000000000030042000FA5B02000000000091
:1034900010042000FA5B020000000000C0042000BD
:1034A000FA5B02000000000090042000FA5B0200BA
:1034B0000000000020042000FA5B02000000000071
:1034C00020052000FA5B020000000000100420002C
:1034D000FA5B02000000000040052000FA5B0200D9
:1034E0000000000090042000FA5B020000000000D1
:1034F000F0042000FA5B020000000000E00420005D
:10350000FA5B020000000000344320006004200049
:103510007C5C020000000000F30F2000030062004A
:10352000FA5B0200000000004822DE000300620097
:10353000FA5B020000000000200420007C5C020016
:1035400000000000D0042000FA5B02000000000030
:10355000F0042000FA5B020000000000400420009C
:10356000FA5B02000000000050042000FA5B020039
:103570000000000084482000600420007C5C020001
:1035800000000000F30F200003006200FA5B02005D
:10359000000000004822DE0003006200FA5B020027
:1035A00000000000200420007C5C020000000000FD
:1035B00000052000FA5B020000000000F00420007B
:1035C000FA5B02000000000070052000FA5B0200B8
:1035D0000000000050042000FA5B02000000000020
:1035E00020052000FA5B020000000000000220001D
:1035F000FA5B020000000000F0042000FA5B020009
:103600000000000060042000FA5B020000000000DF
:1036100060042000FA5B02000000000080382100F6
:10362000E08288002230EC008E0B040000000000D5
:10363000A0C6800031002000010050004220AE00F2
:10364000301B040000000000722102000000000096
:103650002002200010818800A81B04000000000048
:10366000A0C6800011002000010050004220AE00E2
:10367000481B04000000000072210200000000004E
:103680004000200010818800A81B040000000000FA
:10369000A0C6800021002000010050004220AE00A2
:1036A0005C1B040000000000600020001081880006
:1036B000A81B040000000000A0C6800091002000AC
:1036C000010050004220AE00701B0400000000000A
:1036D0008000200010818800A81B0400000000006A
:1036E000A0C6800081002000010050004220AE00F2
:1036F000841B040000000000A0002000108188004E
:10370000A81B040000000000A0C68000710020007B
:10371000010050004220AE00981B04000000000091
:10372000C000200010818800A81B040000000000D9
:103730005C10E2004220AE00A81B04000000000064
:10374000A000200010818800A81B040000000000D9
:103750008E0B040000000000545D02000000000019
:1037600084072000600420007C5C02000000000050
:10377000F30F200003006200FA5B0200000000006B
:103780004822DE0003006200FA5B02000000000035
:10379000200420007C5C02000000000010042000D7
:1037A000FA5B02000000000000072000FA5B020044
:1037B0000000000000072000FA5B0200000000008B
:1037C000C0062000FA5B0200000000009006200006
:1037D000FA5B0200000000000423200060042000C7
:1037E0007C5C020000000000F30F20000300620078
:1037F000FA5B0200000000004822DE0003006200C5
:10380000FA5B020000000000200420007C5C020043
:103810000000000040042000FA5B020000000000ED
:1038200050062000FA5B020000000000E0062000C5
:10383000FA5B02000000000030072000FA5B020083
:103840000000000090062000FA5B0200000000006B
:10385000843E2000600420007C5C02000000000028
:10386000F30F200003006200FA5B0200000000007A
:103870004822DE0003006200FA5B02000000000044
:10388000200420007C5C02000000000020052000D5
:10389000FA5B020000000000F0062000FA5B020064
:1038A0000000000070072000FA5B0200000000002A
:1038B000F0022000FA5B02000000000080042000FB
:1038C000FA5B020000000000B44820006004200001
:1038D0007C5C020000000000F30F20000300620087
:1038E000FA5B0200000000004822DE0003006200D4
:1038F000FA5B020000000000200420007C5C020053
:103900000000000054492000600420007C5C02009C
:1039100000000000F30F200003006200FA5B0200C9
:10392000000000004822DE0003006200FA5B020093
:1039300000000000200420007C5C02000000000069
:10394000044A2000600420007C5C020000000000AB
:10395000F30F200003006200FA5B02000000000089
:103960004822DE0003006200FA5B02000000000053
:10397000200420007C5C020000000000A44A20001B
:10398000600420007C5C020000000000F30F2000B7
:1039900003006200FA5B0200000000004822DE0023
:1039A00003006200FA5B0200000000002004200017
:1039B0007C5C020000000000F44020006004200055
:1039C0007C5C020000000000F30F20000300620096
:1039D000FA5B0200000000004822DE0003006200E3
:1039E000FA5B020000000000200420007C5C020062
:1039F0000000000030052000FA5B0200000000001B
:103A000000072000FA5B02000000000050062000C2
:103A1000FA5B02000000000050062000FA5B020082
:103A20000000000040062000FA5B020000000000D9
:103A300074252000600420007C5C0200000000006F
:103A4000F30F200003006200FA5B02000000000098
:103A50004822DE0003006200FA5B02000000000062
:103A6000200420007C5C02000000000030042000E4
:103A7000FA5B02000000000010062000FA5B020062
:103A800000000000C0062000FA5B020000000000F9
:103A900090062000FA5B02000000000020062000D3
:103AA000FA5B020000000000F4092000600420001E
:103AB0007C5C020000000000F30F200003006200A5
:103AC000FA5B0200000000004822DE0003006200F2
:103AD000FA5B020000000000200420007C5C020071
:103AE0000000000030052000FA5B0200000000002A
:103AF00000072000FA5B0200000000001006200012
:103B0000FA5B02000000000020072000FA5B0200C0
:103B10000000000050062000FA5B020000000000D8
:103B2000B4482000600420007C5C0200000000001B
:103B3000F30F200003006200FA5B020000000000A7
:103B40004822DE0003006200FA5B02000000000071
:103B5000D00520007C5C0200000000004000200036
:103B6000FA5B02000000000070002000FA5B020017
:103B700000000000900520007C5C020000000000B6
:103B800070052000FA5B0200000000002230EC000B
:103B90008E0B04000000000090828000808188006D
:103BA0005662020000000000B48280006004200021
:103BB0007C5C020000000000F30F200003006200A4
:103BC000FA5B0200000000004822DE0003006200F1
:103BD000FA5B020000000000200420007C5C020070
:103BE000000000005082800001032000010040001E
:103BF000FA5B0200000000006082800001032000E8
:103C000001004000FA5B02000000000070828000AA
:103C10000103200001004000FA5B020000000000E8
:103C2000808280000103200001004000FA5B020056
:103C300000000000B4828000C082800000024200C8
:103C4000600420007C5C020000000000F30F2000F4
:103C500003006200FA5B0200000000004822DE0060
:103C600003006200FA5B0200000000005082800046
:103C7000D220020000000000508288005830EC0082
:103C800060828000D2200200000000006082880074
:103C90005830EC0070828000D2200200000000004A
:103CA000708288005830EC0080828000D2200200B0
:103CB000000000008082880084828000A000200034
:103CC000718280000101B80004024100400620001A
:103CD000618280000101B80004024100803E2000A2
:103CE000518280000101B8000402410094828800E2
:103CF00000000600908280008081880056620200E9
:103D000000000000B4828000600420007C5C02009F
:103D100000000000F30F200003006200FA5B0200C5
:103D2000000000004822DE0003006200FA5B02008F
:103D300000000000200420007C5C02000000000065
:103D4000708280000103200001004000FA5B020045
:103D5000000000008082800001032000010040007C
:103D6000FA5B020000000000B4828000C082800084
:103D700000024200600420007C5C020000000000A1
:103D8000F30F200003006200FA5B02000000000055
:103D90004822DE0003006200FA5B0200000000001F
:103DA00070828000D2200200000000007082880033
:103DB0005830EC0080828000D22002000000000019
:103DC0008082880084828000A000200071828000B0
:103DD0000101B8000402410094828800000006003E
:103DE00090828000808188005662020000000000FE
:103DF000B4828000600420007C5C020000000000AF
:103E0000F30F200003006200FA5B020000000000D4
:103E10004822DE0003006200FA5B0200000000009E
:103E2000200420007C5C0200000000006082800012
:103E30000103200001004000FA5B020000000000C6
:103E4000708280000103200001004000FA5B020044
:103E5000000000008082800001032000010040007B
:103E6000FA5B020000000000B4828000C082800083
:103E700000024200600420007C5C020000000000A0
:103E8000F30F200003006200FA5B02000000000054
:103E90004822DE0003006200FA5B0200000000001E
:103EA00060828000D2200200000000006082880052
:103EB0005830EC0070828000D22002000000000028
:103EC000708288005830EC0080828000D22002008E
:103ED000000000008082880084828000A000200012
:103EE000718280000101B8000402410040062000F8
:103EF000618280000101B8000402410094828800C0
:103F000000000600908280008081880056620200D6
:103F100000000000B4828000600420007C5C02008D
:103F200000000000F30F200003006200FA5B0200B3
:103F3000000000004822DE0003006200FA5B02007D
:103F400000000000200420007C5C02000000000053
:103F5000508280000103200001004000FA5B020053
:103F6000000000006082800001032000010040008A
:103F7000FA5B020000000000708280000103200054
:103F800001004000FA5B0200000000008082800017
:103F90000103200001004000FA5B02000000000065
:103FA000B4828000C08280000002420060042000D1
:103FB0007C5C020000000000F30F200003006200A0
:103FC000FA5B0200000000004822DE0003006200ED
:103FD000FA5B02000000000050828000D220020044
:103FE00000000000508288005830EC0060828000A1
:103FF000D220020000000000608288005830EC00EF
:1040000070828000D22002000000000070828800D0
:104010005830EC0080828000D220020000000000B6
:104020008082880084828000A0002000718280004D
:104030000101B800040241004006200061828000B6
:104040000101B80004024100803E2000518280003E
:104050000101B800040241009482880000000600BB
:10406000908280008081880056620200000000007B
:10407000B4828000600420007C5C0200000000002C
:10408000F30F200003006200FA5B02000000000052
:104090004822DE0003006200FA5B0200000000001C
:1040A000200420007C5C02000000000050828000A0
:1040B0000103200001004000FA5B02000000000044
:1040C000E0022000FA5B0200000000006082800035
:1040D0000103200001004000FA5B02000000000024
:1040E000708280000103200001004000FA5B0200A2
:1040F00000000000B4828000C08280000002420004
:10410000600420007C5C020000000000F30F20002F
:1041100003006200FA5B0200000000004822DE009B
:1041200003006200FA5B0200000000005082800081
:10413000D220020000000000508288005830EC00BD
:104140005830EC0060828000D220020000000000A5
:10415000608288005830EC0070828000D22002001B
:10416000000000007082880084828000A00020008F
:10417000718280000101B800040241004006200065
:10418000618280000101B80004024100803E2000ED
:10419000518280000101B80004024100948288002D
:1041A00000000600D0828800B4828000C0828000B7
:1041B00000024200600420007C5C0200000000005D
:1041C000F30F200003006200FA5B02000000000011
:1041D0004822DE0003006200FA5B020000000000DB
:1041E000200420007C5C020000000000D0828000DF
:1041F0000103200001004000FA5B02000000000003
:10420000B4828000C082800000024200600420006E
:104210007C5C020000000000F30F2000030062003D
:10422000FA5B0200000000004822DE00030062008A
:10423000FA5B020000000000A0C6800041002000E0
:10424000010050004220AE003C21040000000000AC
:104250005A30EC00D0828000A10020008100500084
:104260004200AF005A30EF0072210200000000004F
:10427000D420040000000000A0C6800051002000EF
:10428000010050004220AE005E210400000000004A
:104290005A30ED00D0828000A10020009200200062
:1042A000810050004200AF00D282880072210200DB
:1042B00000000000D420040000000000A0C6800020
:1042C00061002000010050004220AE001C210400CB
:1042D000000000007221020000000000D082800077
:1042E00000000600A0C68000F1FF2F000100500072
:1042F0004220AE0072210400000000000000060011
:10430000545D020000000000B4072000600420009B
:104310007C5C020000000000F30F2000030062003C
:10432000FA5B0200000000004822DE000300620089
:10433000FA5B020000000000200420007C5C020008
:104340000000000000052000FA5B020000000000F1
:1043500000022000FA5B020000000000C004200000
:10436000FA5B02000000000000022000FA5B02007D
:104370000000000010042000FA5B020000000000B2
:1043800000022000FA5B020000000000E0042000B0
:10439000FA5B02000000000000022000FA5B02004D
:1043A0000000000040052000FA5B02000000000051
:1043B00000022000FA5B02000000000090042000D0
:1043C000FA5B02000000000000022000FA5B02001D
:1043D00000000000E0042000FA5B02000000000082
:1043E00000022000FA5B02000000000070042000C0
:1043F000FA5B02000000000000022000FA5B0200ED
:104400000000000000022000FA5B02000000000033
:1044100000022000FA5B02000000000030052000CE
:10442000FA5B02000000000000022000FA5B0200BC
:104430000000000050042000FA5B020000000000B1
:1044400000022000FA5B020000000000400520008E
:10445000FA5B02000000000000022000FA5B02008C
:104460000000000040052000FA5B02000000000090
:1044700000022000FA5B020000000000900420000F
:10448000FA5B02000000000000022000FA5B02005C
:1044900000000000E0042000FA5B020000000000C1
:1044A00000022000FA5B02000000000070042000FF
:1044B000FA5B02000000000000022000FA5B02002C
:1044C0000000000030052000FA5B02000000000040
:1044D000340A2000600420007C5C02000000000020
:1044E000F30F200003006200FA5B020000000000EE
:1044F0004822DE0003006200FA5B020000000000B8
:10450000200420007C5C020000000000D00220009B
:10451000FA5B020000000000D0022000FA5B0200FB
:1045200000000000D0022000FA5B02000000000042
:10453000D0022000FA5B020000000000D002200040
:10454000FA5B020000000000D0022000FA5B0200CB
:1045500000000000D0022000FA5B02000000000012
:10456000D0022000FA5B020000000000D002200010
:10457000FA5B020000000000D0022000FA5B02009B
:1045800000000000D0022000FA5B020000000000E2
:10459000D0022000FA5B020000000000D0022000E0
:1045A000FA5B020000000000D0022000FA5B02006B
:1045B00000000000D0022000FA5B020000000000B2
:1045C000D0022000FA5B020000000000D0022000B0
:1045D000FA5B020000000000D0022000FA5B02003B
:1045E00000000000D0022000FA5B02000000000082
:1045F000D0022000FA5B020000000000D002200080
:10460000FA5B020000000000D0022000FA5B02000A
:1046100000000000D0022000FA5B02000000000051
:10462000D0022000FA5B020000000000D00220004F
:10463000FA5B020000000000D0022000FA5B0200DA
:1046400000000000D0022000FA5B02000000000021
:10465000D0022000FA5B020000000000D00220001F
:10466000FA5B020000000000D0022000FA5B0200AA
:1046700000000000D0022000FA5B020000000000F1
:10468000D0022000FA5B020000000000D0022000EF
:10469000FA5B0200000000000423200060042000F8
:1046A0007C5C020000000000F30F200003006200A9
:1046B000FA5B0200000000004822DE0003006200F6
:1046C000FA5B020000000000200420007C5C020075
:1046D0000000000020838000808188005662020074
:1046E0000000000060828000010320000100400003
:1046F000FA5B0200000000007082800001032000CD
:1047000001004000FA5B020000000000808280008F
:104710000103200001004000FA5B020000000000DD
:1047200000022000FA5B020000000000C00420002C
:10473000FA5B02000000000010042000FA5B020097
:1047400000000000E0042000FA5B0200000000000E
:1047500040042000FA5B020000000000000220007C
:10476000FA5B020000000000E0042000FA5B020097
:104770000000000050052000FA5B0200000000006D
:10478000D0042000FA5B020000000000200420009A
:10479000FA5B02000000000050042000FA5B0200F7
:1047A0000000000020052000FA5B0200000000006D
:1047B000843E2000600420007C5C020000000000B9
:1047C000F30F200003006200FA5B0200000000000B
:1047D0004822DE0003006200FA5B020000000000D5
:1047E000200420007C5C02000000000090042000F7
:1047F000FA5B020000000000D0042000FA5B020017
:104800000000000000052000FA5B0200000000002C
:10481000C0042000FA5B02000000000050042000E9
:10482000FA5B020000000000D0042000FA5B0200E6
:104830000000000050042000FA5B020000000000AD
:10484000E0042000FA5B02000000000040052000A8
:10485000FA5B020000000000044120006004200018
:104860007C5C020000000000F30F200003006200E7
:10487000FA5B0200000000004822DE000300620034
:10488000FA5B020000000000200420007C5C0200B3
:104890000000000030052000FA5B0200000000006C
:1048A00050042000FA5B02000000000040052000D8
:1048B000FA5B02000000000040052000FA5B0200E5
:1048C0000000000090042000FA5B020000000000DD
:1048D000E0042000FA5B02000000000070042000E9
:1048E000FA5B02000000000030052000FA5B0200C5
:1048F0000000000084242000600420007C5C020092
:1049000000000000F30F200003006200FA5B0200C9
:10491000000000004822DE0003006200FA5B020093
:1049200000000000200420007C5C02000000000069
:1049300060042000FA5B0200000000005004200028
:10494000FA5B02000000000020052000FA5B020074
:104950000000000040052000FA5B0200000000009B
:1049600090042000FA5B020000000000C004200058
:10497000FA5B02000000000090042000FA5B0200D5
:104980000000000030052000FA5B0200000000007B
:1049900050042000FA5B0200000000002005200007
:1049A000FA5B020000000000642720006004200081
:1049B0007C5C020000000000F30F20000300620096
:1049C000FA5B0200000000004822DE0003006200E3
:1049D000FA5B020000000000200420007C5C020062
:1049E00000000000B0062000FA5B0200000000009A
:1049F00070062000FA5B020000000000F0022000B8
:104A0000FA5B02000000000080062000FA5B020052
:104A10000000000000022000FA5B0200000000001D
:104A20001083800080818800566202000000000030
:104A3000508280000103200001004000FA5B020068
:104A4000000000006082800001032000010040009F
:104A5000FA5B020000000000708280000103200069
:104A600001004000FA5B020000000000808280002C
:104A70000103200001004000FA5B0200000000007A
:104A800004402000600420007C5C02000000000064
:104A9000F30F200003006200FA5B02000000000038
:104AA0004822DE0003006200FA5B02000000000002
:104AB000200420007C5C0200000000006004200054
:104AC000FA5B02000000000050042000FA5B0200C4
:104AD0000000000020052000FA5B0200000000003A
:104AE00040052000FA5B0200000000009004200056
:104AF000FA5B020000000000C0042000FA5B020024
:104B00000000000090042000FA5B0200000000009A
:104B100030052000FA5B0200000000005004200075
:104B2000FA5B02000000000020052000FA5B020092
:104B30000000000004432000600420007C5C0200B0
:104B400000000000F30F200003006200FA5B020087
:104B5000000000004822DE0003006200FA5B020051
:104B600000000000200420007C5C02000000000027
:104B700030052000FA5B02000000000070042000F5
:104B8000FA5B02000000000000022000FA5B020055
:104B900000000000F08080008081880056620200E2
:104BA000000000005082800001032000010040004E
:104BB000FA5B020000000000E0022000FA5B020045
:104BC000000000006082800001032000010040001E
:104BD000FA5B0200000000007082800001032000E8
:104BE00001004000FA5B0200000000008448200041
:104BF000600420007C5C020000000000F30F200035
:104C000003006200FA5B0200000000004822DE00A0
:104C100003006200FA5B0200000000002004200094
:104C20007C5C020000000000D0042000FA5B02005F
:104C30000000000010042000FA5B020000000000E9
:104C400090042000FA5B020000000000E004200055
:104C5000FA5B02000000000000022000FA5B020084
:104C600000000000D0042000FA5B020000000000F9
:104C700050042000FA5B020000000000E004200065
:104C8000FA5B02000000000050052000FA5B020001
:104C90000000000044492000600420007C5C020009
:104CA00000000000F30F200003006200FA5B020026
:104CB000000000004822DE0003006200FA5B0200F0
:104CC00000000000200420007C5C020000000000C6
:104CD00060042000FA5B0200000000009004200045
:104CE000FA5B02000000000020052000FA5B0200D1
:104CF0000000000030052000FA5B02000000000008
:104D000040052000FA5B02000000000000022000C5
:104D1000FA5B02000000000030052000FA5B020090
:104D20000000000050042000FA5B020000000000B8
:104D3000C0042000FA5B02000000000050042000C4
:104D4000FA5B02000000000030042000FA5B020061
:104D50000000000040052000FA5B02000000000097
:104D600000022000FA5B0200000000009004200016
:104D7000FA5B02000000000040052000FA5B020020
:104D80000000000050042000FA5B02000000000058
:104D9000D0042000FA5B02000000000000022000A6
:104DA000FA5B02000000000040052000FA5B0200F0
:104DB00000000000F0042000FA5B02000000000088
:104DC00000022000FA5B0200000000001004200036
:104DD000FA5B02000000000040042000FA5B0200C1
:104DE00000000000A0042000FA5B020000000000A8
:104DF00050052000FA5B0200000000003005200092
:104E0000FA5B02000000000040052000FA5B02008F
:104E10000000000000712200E08288009000200065
:104E2000108188008E0B040000000000A0C68000E6
:104E300031002000010050004220AE005227040043
:104E4000000000007221020000000000007122003A
:104E500080818800000020009081880000002000F0
:104E6000A081880050838000B0818800000020006D
:104E7000C081880000002000D0818800186A0200EC
:104E800000000000808180000081880042730200E1
:104E9000000000002000200010818800C2270400CC
:104EA00000000000A0C6800011002000010050009A
:104EB0004220AE006A2704000000000072210200B8
:104EC00000000000E000200010818800C2270400DC
:104ED00000000000A0C6800021002000010050005A
:104EE0004220AE0082270400000000007221020070
:104EF000000000000001200010818800C22704008B
:104F000000000000A0C680008100200001005000C9
:104F10004220AE009A270400000000007221020027
:104F2000000000002001200010818800C22704003A
:104F300000000000A0C680007100200001005000A9
:104F40004220AE00B22704000000000072210200DF
:104F5000000000004001200010818800C2270400EA
:104F6000000000005C10E2004220AE00C2270400F6
:104F7000000000002000200010818800C2270400EB
:104F8000000000008E0B0400000000008448200098
:104F9000600420007C5C020000000000F30F200091
:104FA00003006200FA5B0200000000004822DE00FD
:104FB00003006200FA5B02000000000020042000F1
:104FC0007C5C02000000000000022000FA5B02008E
:104FD0000000000000022000FA5B02000000000058
:104FE00000022000FA5B0200000000000002200026
:104FF000FA5B02000000000000022000FA5B0200E1
:105000000000000000022000FA5B02000000000027
:1050100000022000FA5B02000000000000022000F5
:10502000FA5B02000000000000022000FA5B0200B0
:105030000000000044492000600420007C5C020065
:1050400000000000F30F200003006200FA5B020082
:10505000000000004822DE0003006200FA5B02004C
:1050600000000000200420007C5C02000000000022
:1050700000022000FA5B0200000000000002200095
:10508000FA5B02000000000050052000FA5B0200FD
:105090000000000000052000FA5B02000000000094
:1050A00000022000FA5B0200000000000002200065
:1050B000FA5B02000000000000022000FA5B020020
:1050C0000000000000022000FA5B02000000000067
:1050D00000022000FA5B0200000000000002200035
:1050E000FA5B02000000000000022000FA5B0200F0
:1050F0000000000000022000FA5B02000000000037
:1051000040042000FA5B020000000000F0042000D0
:10511000FA5B02000000000070052000FA5B02004C
:1051200000000000E0042000FA5B02000000000024
:1051300000022000FA5B02000000000000022000D4
:10514000FA5B02000000000000022000FA5B02008F
:105150000000000000022000FA5B020000000000D6
:1051600000022000FA5B02000000000000022000A4
:10517000FA5B02000000000030052000FA5B02002C
:105180000000000040052000FA5B02000000000063
:10519000F0042000FA5B020000000000200520005F
:1051A000FA5B02000000000050042000FA5B0200DD
:1051B00000000000F0002000108188008E0B040029
:1051C00000000000208380009082880000232000DF
:1051D000B082880000002000C0828800F01E02001B
:1051E0000000000090828000208388008448200016
:1051F000600420007C5C020000000000F30F20002F
:1052000003006200FA5B0200000000004822DE009A
:1052100003006200FA5B020000000000200420008E
:105220007C5C020000000000D0042000FA5B020059
:105230000000000010042000FA5B020000000000E3
:1052400090042000FA5B020000000000E00420004F
:10525000FA5B02000000000000022000FA5B02007E
:1052600000000000D0042000FA5B020000000000F3
:1052700050042000FA5B020000000000E00420005F
:10528000FA5B02000000000050052000FA5B0200FB
:105290000000000044492000600420007C5C020003
:1052A00000000000F30F200003006200FA5B020020
:1052B000000000004822DE0003006200FA5B0200EA
:1052C00000000000200420007C5C020000000000C0
:1052D00060042000FA5B020000000000900420003F
:1052E000FA5B02000000000020052000FA5B0200CB
:1052F0000000000030052000FA5B02000000000002
:1053000040052000FA5B02000000000000022000BF
:10531000FA5B02000000000030052000FA5B02008A
:105320000000000050042000FA5B020000000000B2
:10533000C0042000FA5B02000000000050042000BE
:10534000FA5B02000000000030042000FA5B02005B
:105350000000000040052000FA5B02000000000091
:1053600000022000FA5B0200000000009004200010
:10537000FA5B02000000000040052000FA5B02001A
:105380000000000050042000FA5B02000000000052
:10539000D0042000FA5B02000000000000022000A0
:1053A000FA5B02000000000040052000FA5B0200EA
:1053B00000000000F0042000FA5B02000000000082
:1053C00000022000FA5B0200000000001004200030
:1053D000FA5B02000000000040042000FA5B0200BB
:1053E00000000000A0042000FA5B020000000000A2
:1053F00050052000FA5B020000000000300520008C
:10540000FA5B02000000000040052000FA5B020089
:105410000000000000712200E0828800900020005F
:10542000108188008E0B04000000000084482000DA
:10543000600420007C5C020000000000F30F2000EC
:1054400003006200FA5B0200000000004822DE0058
:1054500003006200FA5B020000000000200420004C
:105460007C5C02000000000000022000FA5B0200E9
:105470000000000000022000FA5B020000000000B3
:1054800000022000FA5B0200000000000002200081
:10549000FA5B02000000000000022000FA5B02003C
:1054A0000000000000022000FA5B02000000000083
:1054B00000022000FA5B0200000000000002200051
:1054C000FA5B02000000000000022000FA5B02000C
:1054D0000000000044492000600420007C5C0200C1
:1054E00000000000F30F200003006200FA5B0200DE
:1054F000000000004822DE0003006200FA5B0200A8
:1055000000000000200420007C5C0200000000007D
:1055100000022000FA5B02000000000000022000F0
:10552000FA5B02000000000050052000FA5B020058
:105530000000000000052000FA5B020000000000EF
:1055400000022000FA5B02000000000000022000C0
:10555000FA5B02000000000000022000FA5B02007B
:105560000000000000022000FA5B020000000000C2
:1055700000022000FA5B0200000000000002200090
:10558000FA5B02000000000000022000FA5B02004B
:105590000000000000022000FA5B02000000000092
:1055A00040042000FA5B020000000000F00420002C
:1055B000FA5B02000000000070052000FA5B0200A8
:1055C00000000000E0042000FA5B02000000000080
:1055D00000022000FA5B0200000000000002200030
:1055E000FA5B02000000000000022000FA5B0200EB
:1055F0000000000000022000FA5B02000000000032
:1056000000022000FA5B02000000000000022000FF
:10561000FA5B02000000000030052000FA5B020087
:105620000000000040052000FA5B020000000000BE
:10563000F0042000FA5B02000000000020052000BA
:10564000FA5B02000000000050042000FA5B020038
:105650000000000030012000108188008E0B040043
:10566000000000001083800090828800B027200096
:10567000B082880000002000C0828800821F0200E3
:105680000000000090828000108388008448200081
:10569000600420007C5C020000000000F30F20008A
:1056A00003006200FA5B0200000000004822DE00F6
:1056B00003006200FA5B02000000000020042000EA
:1056C0007C5C020000000000D0042000FA5B0200B5
:1056D0000000000010042000FA5B0200000000003F
:1056E00090042000FA5B020000000000E0042000AB
:1056F000FA5B02000000000000022000FA5B0200DA
:1057000000000000D0042000FA5B0200000000004E
:1057100050042000FA5B020000000000E0042000BA
:10572000FA5B02000000000050052000FA5B020056
:105730000000000044492000600420007C5C02005E
:1057400000000000F30F200003006200FA5B02007B
:10575000000000004822DE0003006200FA5B020045
:1057600000000000200420007C5C0200000000001B
:1057700060042000FA5B020000000000900420009A
:10578000FA5B02000000000020052000FA5B020026
:105790000000000030052000FA5B0200000000005D
:1057A00040052000FA5B020000000000000220001B
:1057B000FA5B02000000000030052000FA5B0200E6
:1057C0000000000050042000FA5B0200000000000E
:1057D000C0042000FA5B020000000000500420001A
:1057E000FA5B02000000000030042000FA5B0200B7
:1057F0000000000040052000FA5B020000000000ED
:1058000000022000FA5B020000000000900420006B
:10581000FA5B02000000000040052000FA5B020075
:105820000000000050042000FA5B020000000000AD
:10583000D0042000FA5B02000000000000022000FB
:10584000FA5B02000000000040052000FA5B020045
:1058500000000000F0042000FA5B020000000000DD
:1058600000022000FA5B020000000000100420008B
:10587000FA5B02000000000040042000FA5B020016
:1058800000000000A0042000FA5B020000000000FD
:1058900050052000FA5B02000000000030052000E7
:1058A000FA5B02000000000040052000FA5B0200E5
:1058B0000000000000712200E082880090002000BB
:1058C000108188008E0B0400000000008448200036
:1058D000600420007C5C020000000000F30F200048
:1058E00003006200FA5B0200000000004822DE00B4
:1058F00003006200FA5B02000000000020042000A8
:105900007C5C02000000000000022000FA5B020044
:105910000000000000022000FA5B0200000000000E
:1059200000022000FA5B02000000000000022000DC
:10593000FA5B02000000000000022000FA5B020097
:105940000000000000022000FA5B020000000000DE
:1059500000022000FA5B02000000000000022000AC
:10596000FA5B02000000000000022000FA5B020067
:105970000000000044492000600420007C5C02001C
:1059800000000000F30F200003006200FA5B020039
:10599000000000004822DE0003006200FA5B020003
:1059A00000000000200420007C5C020000000000D9
:1059B00000022000FA5B020000000000000220004C
:1059C000FA5B02000000000050052000FA5B0200B4
:1059D0000000000000052000FA5B0200000000004B
:1059E00000022000FA5B020000000000000220001C
:1059F000FA5B02000000000000022000FA5B0200D7
:105A00000000000000022000FA5B0200000000001D
:105A100000022000FA5B02000000000000022000EB
:105A2000FA5B02000000000000022000FA5B0200A6
:105A30000000000000022000FA5B020000000000ED
:105A400040042000FA5B020000000000F004200087
:105A5000FA5B02000000000070052000FA5B020003
:105A600000000000E0042000FA5B020000000000DB
:105A700000022000FA5B020000000000000220008B
:105A8000FA5B02000000000000022000FA5B020046
:105A90000000000000022000FA5B0200000000008D
:105AA00000022000FA5B020000000000000220005B
:105AB000FA5B02000000000030052000FA5B0200E3
:105AC0000000000040052000FA5B0200000000001A
:105AD000F0042000FA5B0200000000002005200016
:105AE000FA5B02000000000050042000FA5B020094
:105AF0000000000050012000108188008E0B04007F
:105B000000000000F0808000908288003043200078
:105B1000B082880000002000C0828800302002008F
:105B20000000000090828000F080880084482000FF
:105B3000600420007C5C020000000000F30F2000E5
:105B400003006200FA5B0200000000004822DE0051
:105B500003006200FA5B0200000000002004200045
:105B60007C5C020000000000D0042000FA5B020010
:105B70000000000010042000FA5B0200000000009A
:105B800090042000FA5B020000000000E004200006
:105B9000FA5B02000000000000022000FA5B020035
:105BA00000000000D0042000FA5B020000000000AA
:105BB00050042000FA5B020000000000E004200016
:105BC000FA5B02000000000050052000FA5B0200B2
:105BD0000000000044492000600420007C5C0200BA
:105BE00000000000F30F200003006200FA5B0200D7
:105BF000000000004822DE0003006200FA5B0200A1
:105C000000000000200420007C5C02000000000076
:105C100060042000FA5B02000000000090042000F5
:105C2000FA5B02000000000020052000FA5B020081
:105C30000000000030052000FA5B020000000000B8
:105C400040052000FA5B0200000000000002200076
:105C5000FA5B02000000000030052000FA5B020041
:105C60000000000050042000FA5B02000000000069
:105C7000C0042000FA5B0200000000005004200075
:105C8000FA5B02000000000030042000FA5B020012
:105C90000000000040052000FA5B02000000000048
:105CA00000022000FA5B02000000000090042000C7
:105CB000FA5B02000000000040052000FA5B0200D1
:105CC0000000000050042000FA5B02000000000009
:105CD000D0042000FA5B0200000000000002200057
:105CE000FA5B02000000000040052000FA5B0200A1
:105CF00000000000F0042000FA5B02000000000039
:105D000000022000FA5B02000000000010042000E6
:105D1000FA5B02000000000040042000FA5B020071
:105D200000000000A0042000FA5B02000000000058
:105D300050052000FA5B0200000000003005200042
:105D4000FA5B02000000000040052000FA5B020040
:105D50000000000000712200E08288009000200016
:105D6000108188008E0B040000000000545D0200CA
:105D700000000000B4082000600420007C5C0200E9
:105D800000000000F30F200003006200FA5B020035
:105D9000000000004822DE0003006200FA5B0200FF
:105DA00000000000200420007C5C020000000000D5
:105DB00090042000FA5B02000000000000022000B6
:105DC000FA5B020000000000D0042000FA5B020031
:105DD0000000000000022000FA5B0200000000004A
:105DE00000052000FA5B0200000000000002200015
:105DF000FA5B020000000000C0042000FA5B020011
:105E00000000000000022000FA5B02000000000019
:105E100050042000FA5B0200000000000002200095
:105E2000FA5B020000000000D0042000FA5B0200D0
:105E30000000000000022000FA5B020000000000E9
:105E400050042000FA5B0200000000000002200065
:105E5000FA5B020000000000E0042000FA5B020090
:105E60000000000000022000FA5B020000000000B9
:105E700040052000FA5B020000000000340B200007
:105E8000600420007C5C020000000000F30F200092
:105E900003006200FA5B0200000000004822DE00FE
:105EA00003006200FA5B02000000000020042000F2
:105EB0007C5C020000000000D0022000FA5B0200BF
:105EC00000000000D0022000FA5B02000000000089
:105ED000D0022000FA5B020000000000D002200087
:105EE000FA5B020000000000D0022000FA5B020012
:105EF00000000000D0022000FA5B02000000000059
:105F0000D0022000FA5B020000000000D002200056
:105F1000FA5B020000000000D0022000FA5B0200E1
:105F200000000000D0022000FA5B02000000000028
:105F3000D0022000FA5B020000000000D002200026
:105F4000FA5B020000000000D0022000FA5B0200B1
:105F500000000000D0022000FA5B020000000000F8
:105F6000D0022000FA5B020000000000D0022000F6
:105F7000FA5B020000000000D0022000FA5B020081
:105F80000000000044102000600420007C5C02003F
:105F900000000000F30F200003006200FA5B020023
:105FA000000000004822DE0003006200FA5B0200ED
:105FB00000000000200420007C5C020000000000C3
:105FC00030052000FA5B0200000000000002200003
:105FD000FA5B02000000000050042000FA5B02009F
:105FE0000000000000022000FA5B02000000000038
:105FF00040052000FA5B02000000000000022000C3
:10600000FA5B02000000000040052000FA5B02007D
:106010000000000000022000FA5B02000000000007
:1060200090042000FA5B0200000000000002200043
:10603000FA5B020000000000E0042000FA5B0200AE
:106040000000000000022000FA5B020000000000D7
:1060500070042000FA5B0200000000000002200033
:10606000FA5B02000000000030052000FA5B02002D
:1060700000000000C4122000600420007C5C0200CC
:1060800000000000F30F200003006200FA5B020032
:10609000000000004822DE0003006200FA5B0200FC
:1060A00000000000200420007C5C020000000000D2
:1060B000D0022000FA5B020000000000D0022000A5
:1060C000FA5B020000000000D0022000FA5B020030
:1060D00000000000D0022000FA5B02000000000077
:1060E000D0022000FA5B020000000000D002200075
:1060F000FA5B020000000000D0022000FA5B020000
:1061000000000000D0022000FA5B02000000000046
:10611000D0022000FA5B020000000000D002200044
:10612000FA5B020000000000D0022000FA5B0200CF
:1061300000000000D0022000FA5B02000000000016
:10614000D0022000FA5B020000000000D002200014
:10615000FA5B020000000000D0022000FA5B02009F
:106160000000000084072000600420007C5C020026
:1061700000000000F30F200003006200FA5B020041
:10618000000000004822DE0003006200FA5B02000B
:1061900000000000200420007C5C020000000000E1
:1061A0003083800080818800566202000000000079
:1061B000708280000103200001004000FA5B0200B1
:1061C00000000000808280000103200001004000E8
:1061D000FA5B02000000000000022000FA5B0200EF
:1061E0000000000090042000FA5B020000000000A4
:1061F000E0022000FA5B02000000000040042000E2
:10620000FA5B020000000000E0022000FA5B0200DE
:106210000000000000022000FA5B02000000000005
:10622000E0042000FA5B020000000000F0062000FD
:10623000FA5B02000000000004232000600420003C
:106240007C5C020000000000F30F200003006200ED
:10625000FA5B0200000000004822DE00030062003A
:10626000FA5B020000000000200420007C5C0200B9
:106270000000000040838000808188005662020098
:106280000000000070828000010320000100400037
:10629000FA5B020000000000808280000103200001
:1062A00001004000FA5B0200000000000002200034
:1062B000FA5B020000000000E0042000FA5B02002C
:1062C00000000000F0062000FA5B02000000000061
:1062D00000022000FA5B020000000000F004200031
:1062E000FA5B02000000000060042000FA5B02007C
:1062F0000000000000022000FA5B02000000000025
:1063000020052000FA5B020000000000F0042000DD
:10631000FA5B02000000000070052000FA5B02003A
:106320000000000030052000FA5B020000000000C1
:10633000843E2000600420007C5C0200000000001D
:10634000F30F200003006200FA5B0200000000006F
:106350004822DE0003006200FA5B02000000000039
:10636000200420007C5C02000000000050838000BC
:106370008081880056620200000000006082800078
:106380000103200001004000FA5B02000000000051
:10639000708280000103200001004000FA5B0200CF
:1063A0000000000080828000010320000100400006
:1063B000FA5B02000000000000022000FA5B02000D
:1063C0000000000020052000FA5B02000000000031
:1063D000F0042000FA5B02000000000070052000BD
:1063E000FA5B02000000000000022000FA5B0200DD
:1063F0000000000070052000FA5B020000000000B1
:1064000090042000FA5B020000000000400420001D
:10641000FA5B02000000000040052000FA5B020069
:106420000000000080042000FA5B02000000000071
:1064300000022000FA5B020000000000300620008D
:10644000FA5B020000000000D0062000FA5B0200A8
:106450000000000014242000600420007C5C020086
:1064600000000000F30F200003006200FA5B02004E
:10647000000000004822DE0003006200FA5B020018
:1064800000000000200420007C5C020000000000EE
:1064900000052000FA5B020000000000C00420009C
:1064A000FA5B02000000000010042000FA5B02000A
:1064B00000000000E0042000FA5B02000000000081
:1064C00040052000FA5B020000000000500420009C
:1064D000FA5B02000000000020052000FA5B0200C9
:1064E0000000000000022000FA5B02000000000033
:1064F000F0022000FA5B0200000000000002200011
:10650000FA5B02000000000030042000FA5B020089
:106510000000000050052000FA5B020000000000AF
:10652000C0042000FA5B02000000000040052000CB
:10653000FA5B02000000000090042000FA5B0200F9
:106540000000000060052000FA5B0200000000006F
:1065500010042000FA5B020000000000400520004B
:10656000FA5B020000000000F0042000FA5B020069
:106570000000000020052000FA5B0200000000007F
:1065800000022000FA5B020000000000608380002F
:10659000FA5B020000000000D43F200060042000ED
:1065A0007C5C020000000000F30F2000030062008A
:1065B000FA5B0200000000004822DE0003006200D7
:1065C000FA5B020000000000200420007C5C020056
:1065D0000000000040052000FA5B020000000000FF
:1065E00010042000FA5B020000000000E00420001C
:1065F000FA5B020000000000B0042000FA5B020019
:106600000000000000022000FA5B02000000000011
:1066100030042000FA5B020000000000100420009B
:10662000FA5B02000000000000052000FA5B020097
:106630000000000010042000FA5B020000000000CF
:1066400030042000FA5B02000000000090042000EB
:10665000FA5B02000000000040052000FA5B020027
:106660000000000090052000FA5B0200000000001E
:1066700000022000FA5B020000000000C44220007B
:10668000600420007C5C020000000000F30F20008A
:1066900003006200FA5B0200000000004822DE00F6
:1066A00003006200FA5B02000000000020042000EA
:1066B0007C5C020000000000C0042000FA5B0200C5
:1066C0000000000090042000FA5B020000000000BF
:1066D00040052000FA5B02000000000020052000B9
:1066E000FA5B02000000000050042000FA5B020088
:1066F0000000000030052000FA5B020000000000EE
:1067000000022000FA5B020000000000708380009D
:1067100080818800566202000000000050828000E4
:106720000103200001004000FA5B020000000000AD
:10673000608280000103200001004000FA5B02003B
:106740000000000070828000010320000100400072
:10675000FA5B02000000000080828000010320003C
:1067600001004000FA5B02000000000084482000A5
:10677000600420007C5C020000000000F30F200099
:1067800003006200FA5B0200000000004822DE0005
:1067900003006200FA5B02000000000020042000F9
:1067A0007C5C02000000000000022000FA5B020096
:1067B0000000000000022000FA5B02000000000060
:1067C00000022000FA5B020000000000200420000C
:1067D000FA5B02000000000010042000FA5B0200D7
:1067E0000000000030042000FA5B020000000000FE
:1067F000B0042000FA5B020000000000000220004C
:10680000FA5B02000000000000022000FA5B0200B8
:106810000000000044492000600420007C5C02006D
:1068200000000000F30F200003006200FA5B02008A
:10683000000000004822DE0003006200FA5B020054
:1068400000000000200420007C5C0200000000002A
:1068500060042000FA5B02000000000090042000A9
:10686000FA5B02000000000020052000FA5B020035
:106870000000000030052000FA5B0200000000006C
:1068800040052000FA5B020000000000000220002A
:10689000FA5B02000000000030052000FA5B0200F5
:1068A0000000000050042000FA5B0200000000001D
:1068B000C0042000FA5B0200000000005004200029
:1068C000FA5B02000000000030042000FA5B0200C6
:1068D0000000000040052000FA5B020000000000FC
:1068E00000022000FA5B020000000000900420007B
:1068F000FA5B02000000000040052000FA5B020085
:106900000000000050042000FA5B020000000000BC
:10691000D0042000FA5B020000000000000220000A
:10692000FA5B02000000000040052000FA5B020054
:1069300000000000F0042000FA5B020000000000EC
:1069400000022000FA5B020000000000100420009A
:10695000FA5B02000000000040042000FA5B020025
:1069600000000000A0042000FA5B0200000000000C
:1069700050052000FA5B02000000000030052000F6
:10698000FA5B02000000000040052000FA5B0200F4
:106990000000000000712200E08288001001200049
:1069A000108188008E0B040000000000A0C680004B
:1069B00031002000010050004220AE00EE340400FF
:1069C0000000000072210200000000008000200092
:1069D000108188007635040000000000A0C6800009
:1069E00001002000010050004220AE0006350400E6
:1069F0000000000072210200000000006001200081
:106A0000108188007635040000000000A0C68000D8
:106A100011002000010050004220AE001E3504008D
:106A20000000000072210200000000008001200030
:106A3000108188007635040000000000A0C68000A8
:106A400021002000010050004220AE003635040035
:106A5000000000007221020000000000A0012000E0
:106A6000108188007635040000000000A0C6800078
:106A700081002000010050004220AE004E3504008D
:106A8000000000007221020000000000C001200090
:106A9000108188007635040000000000A0C6800048
:106AA00071002000010050004220AE006635040055
:106AB000000000007221020000000000E001200040
:106AC0001081880076350400000000005C10E200B0
:106AD0004220AE0076350400000000008000200057
:106AE0001081880076350400000000008E0B040041
:106AF0000000000084482000600420007C5C02004C
:106B000000000000F30F200003006200FA5B0200A7
:106B1000000000004822DE0003006200FA5B020071
:106B200000000000200420007C5C02000000000047
:106B300000022000FA5B02000000000000022000BA
:106B4000FA5B02000000000000022000FA5B020075
:106B50000000000000022000FA5B020000000000BC
:106B600000022000FA5B020000000000000220008A
:106B7000FA5B02000000000000022000FA5B020045
:106B80000000000000022000FA5B0200000000008C
:106B900000022000FA5B02000000000044492000CF
:106BA000600420007C5C020000000000F30F200065
:106BB00003006200FA5B0200000000004822DE00D1
:106BC00003006200FA5B02000000000020042000C5
:106BD0007C5C02000000000000022000FA5B020062
:106BE0000000000000022000FA5B0200000000002C
:106BF00050052000FA5B02000000000000052000A4
:106C0000FA5B02000000000000022000FA5B0200B4
:106C10000000000000022000FA5B020000000000FB
:106C200000022000FA5B02000000000000022000C9
:106C3000FA5B02000000000000022000FA5B020084
:106C40000000000000022000FA5B020000000000CB
:106C500000022000FA5B0200000000000002200099
:106C6000FA5B02000000000040042000FA5B020012
:106C700000000000F0042000FA5B020000000000A9
:106C800070052000FA5B020000000000E004200014
:106C9000FA5B02000000000000022000FA5B020024
:106CA0000000000000022000FA5B0200000000006B
:106CB00000022000FA5B0200000000000002200039
:106CC000FA5B02000000000000022000FA5B0200F4
:106CD0000000000000022000FA5B0200000000003B
:106CE00030052000FA5B0200000000004005200093
:106CF000FA5B020000000000F0042000FA5B0200D2
:106D00000000000020052000FA5B020000000000E7
:106D100050042000FA5B0200000000007001200017
:106D2000108188008E0B040000000000308380007A
:106D30009082880080072000B08288000000200038
:106D4000C08288007A1E020000000000908280004D
:106D50003083880084482000600420007C5C0200AE
:106D600000000000F30F200003006200FA5B020045
:106D7000000000004822DE0003006200FA5B02000F
:106D800000000000200420007C5C020000000000E5
:106D900000022000FA5B0200000000000002200058
:106DA000FA5B02000000000000022000FA5B020013
:106DB0000000000020042000FA5B02000000000038
:106DC00010042000FA5B02000000000030042000E4
:106DD000FA5B020000000000B0042000FA5B020031
:106DE0000000000000022000FA5B0200000000002A
:106DF00000022000FA5B020000000000444920006D
:106E0000600420007C5C020000000000F30F200002
:106E100003006200FA5B0200000000004822DE006E
:106E200003006200FA5B0200000000002004200062
:106E30007C5C02000000000060042000FA5B02009D
:106E40000000000090042000FA5B02000000000037
:106E500020052000FA5B0200000000003005200041
:106E6000FA5B02000000000040052000FA5B02000F
:106E70000000000000022000FA5B02000000000099
:106E800030052000FA5B02000000000050042000E2
:106E9000FA5B020000000000C0042000FA5B020060
:106EA0000000000050042000FA5B02000000000017
:106EB00030042000FA5B02000000000040052000C2
:106EC000FA5B02000000000000022000FA5B0200F2
:106ED0000000000090042000FA5B020000000000A7
:106EE00040052000FA5B0200000000005004200072
:106EF000FA5B020000000000D0042000FA5B0200F0
:106F00000000000000022000FA5B02000000000008
:106F100040052000FA5B020000000000F0042000A1
:106F2000FA5B02000000000000022000FA5B020091
:106F30000000000010042000FA5B020000000000C6
:106F400040042000FA5B020000000000A0042000C2
:106F5000FA5B02000000000050052000FA5B02000E
:106F60000000000030052000FA5B02000000000075
:106F700040052000FA5B02000000000000712200C2
:106F8000E082880010012000108188008E0B040030
:106F90000000000084482000600420007C5C0200A7
:106FA00000000000F30F200003006200FA5B020003
:106FB000000000004822DE0003006200FA5B0200CD
:106FC00000000000200420007C5C020000000000A3
:106FD00000022000FA5B0200000000000002200016
:106FE000FA5B02000000000000022000FA5B0200D1
:106FF0000000000000022000FA5B02000000000018
:1070000000022000FA5B02000000000000022000E5
:10701000FA5B02000000000000022000FA5B0200A0
:107020000000000000022000FA5B020000000000E7
:1070300000022000FA5B020000000000444920002A
:10704000600420007C5C020000000000F30F2000C0
:1070500003006200FA5B0200000000004822DE002C
:1070600003006200FA5B0200000000002004200020
:107070007C5C02000000000000022000FA5B0200BD
:107080000000000000022000FA5B02000000000087
:1070900050052000FA5B02000000000000052000FF
:1070A000FA5B02000000000000022000FA5B020010
:1070B0000000000000022000FA5B02000000000057
:1070C00000022000FA5B0200000000000002200025
:1070D000FA5B02000000000000022000FA5B0200E0
:1070E0000000000000022000FA5B02000000000027
:1070F00000022000FA5B02000000000000022000F5
:10710000FA5B02000000000040042000FA5B02006D
:1071100000000000F0042000FA5B02000000000004
:1071200070052000FA5B020000000000E00420006F
:10713000FA5B02000000000000022000FA5B02007F
:107140000000000000022000FA5B020000000000C6
:1071500000022000FA5B0200000000000002200094
:10716000FA5B02000000000000022000FA5B02004F
:107170000000000000022000FA5B02000000000096
:1071800030052000FA5B02000000000040052000EE
:10719000FA5B020000000000F0042000FA5B02002D
:1071A0000000000020052000FA5B02000000000043
:1071B00050042000FA5B0200000000009001200053
:1071C000108188008E0B04000000000040838000C6
:1071D0009082880000232000B082880000002000F8
:1071E000C08288007A1E02000000000090828000A9
:1071F0004083880084482000600420007C5C0200FA
:1072000000000000F30F200003006200FA5B0200A0
:10721000000000004822DE0003006200FA5B02006A
:1072200000000000200420007C5C02000000000040
:1072300000022000FA5B02000000000000022000B3
:10724000FA5B02000000000000022000FA5B02006E
:107250000000000020042000FA5B02000000000093
:1072600010042000FA5B020000000000300420003F
:10727000FA5B020000000000B0042000FA5B02008C
:107280000000000000022000FA5B02000000000085
:1072900000022000FA5B02000000000044492000C8
:1072A000600420007C5C020000000000F30F20005E
:1072B00003006200FA5B0200000000004822DE00CA
:1072C00003006200FA5B02000000000020042000BE
:1072D0007C5C02000000000060042000FA5B0200F9
:1072E0000000000090042000FA5B02000000000093
:1072F00020052000FA5B020000000000300520009D
:10730000FA5B02000000000040052000FA5B02006A
:107310000000000000022000FA5B020000000000F4
:1073200030052000FA5B020000000000500420003D
:10733000FA5B020000000000C0042000FA5B0200BB
:107340000000000050042000FA5B02000000000072
:1073500030042000FA5B020000000000400520001D
:10736000FA5B02000000000000022000FA5B02004D
:107370000000000090042000FA5B02000000000002
:1073800040052000FA5B02000000000050042000CD
:10739000FA5B020000000000D0042000FA5B02004B
:1073A0000000000000022000FA5B02000000000064
:1073B00040052000FA5B020000000000F0042000FD
:1073C000FA5B02000000000000022000FA5B0200ED
:1073D0000000000010042000FA5B02000000000022
:1073E00040042000FA5B020000000000A00420001E
:1073F000FA5B02000000000050052000FA5B02006A
:107400000000000030052000FA5B020000000000D0
:1074100040052000FA5B020000000000007122001D
:10742000E082880010012000108188008E0B04008B
:107430000000000084482000600420007C5C020002
:1074400000000000F30F200003006200FA5B02005E
:10745000000000004822DE0003006200FA5B020028
:1074600000000000200420007C5C020000000000FE
:1074700000022000FA5B0200000000000002200071
:10748000FA5B02000000000000022000FA5B02002C
:107490000000000000022000FA5B02000000000073
:1074A00000022000FA5B0200000000000002200041
:1074B000FA5B02000000000000022000FA5B0200FC
:1074C0000000000000022000FA5B02000000000043
:1074D00000022000FA5B0200000000004449200086
:1074E000600420007C5C020000000000F30F20001C
:1074F00003006200FA5B0200000000004822DE0088
:1075000003006200FA5B020000000000200420007B
:107510007C5C02000000000000022000FA5B020018
:107520000000000000022000FA5B020000000000E2
:1075300050052000FA5B020000000000000520005A
:10754000FA5B02000000000000022000FA5B02006B
:107550000000000000022000FA5B020000000000B2
:1075600000022000FA5B0200000000000002200080
:10757000FA5B02000000000000022000FA5B02003B
:107580000000000000022000FA5B02000000000082
:1075900000022000FA5B0200000000000002200050
:1075A000FA5B02000000000040042000FA5B0200C9
:1075B00000000000F0042000FA5B02000000000060
:1075C00070052000FA5B020000000000E0042000CB
:1075D000FA5B02000000000000022000FA5B0200DB
:1075E0000000000000022000FA5B02000000000022
:1075F00000022000FA5B02000000000000022000F0
:10760000FA5B02000000000000022000FA5B0200AA
:107610000000000000022000FA5B020000000000F1
:1076200030052000FA5B0200000000004005200049
:10763000FA5B020000000000F0042000FA5B020088
:107640000000000020052000FA5B0200000000009E
:1076500050042000FA5B020000000000B00120008E
:10766000108188008E0B0400000000005083800011
:1076700090828800803E2000B082880000002000B8
:10768000C0828800F01E020000000000908280008E
:107690005083880084482000600420007C5C020045
:1076A00000000000F30F200003006200FA5B0200FC
:1076B000000000004822DE0003006200FA5B0200C6
:1076C00000000000200420007C5C0200000000009C
:1076D00000022000FA5B020000000000000220000F
:1076E000FA5B02000000000000022000FA5B0200CA
:1076F0000000000020042000FA5B020000000000EF
:1077000010042000FA5B020000000000300420009A
:10771000FA5B020000000000B0042000FA5B0200E7
:107720000000000000022000FA5B020000000000E0
:1077300000022000FA5B0200000000004449200023
:10774000600420007C5C020000000000F30F2000B9
:1077500003006200FA5B0200000000004822DE0025
:1077600003006200FA5B0200000000002004200019
:107770007C5C02000000000060042000FA5B020054
:107780000000000090042000FA5B020000000000EE
:1077900020052000FA5B02000000000030052000F8
:1077A000FA5B02000000000040052000FA5B0200C6
:1077B0000000000000022000FA5B02000000000050
:1077C00030052000FA5B0200000000005004200099
:1077D000FA5B020000000000C0042000FA5B020017
:1077E0000000000050042000FA5B020000000000CE
:1077F00030042000FA5B0200000000004005200079
:10780000FA5B02000000000000022000FA5B0200A8
:107810000000000090042000FA5B0200000000005D
:1078200040052000FA5B0200000000005004200028
:10783000FA5B020000000000D0042000FA5B0200A6
:107840000000000000022000FA5B020000000000BF
:1078500040052000FA5B020000000000F004200058
:10786000FA5B02000000000000022000FA5B020048
:107870000000000010042000FA5B0200000000007D
:1078800040042000FA5B020000000000A004200079
:10789000FA5B02000000000050052000FA5B0200C5
:1078A0000000000030052000FA5B0200000000002C
:1078B00040052000FA5B0200000000000071220079
:1078C000E082880010012000108188008E0B0400E7
:1078D0000000000084482000600420007C5C02005E
:1078E00000000000F30F200003006200FA5B0200BA
:1078F000000000004822DE0003006200FA5B020084
:1079000000000000200420007C5C02000000000059
:1079100000022000FA5B02000000000000022000CC
:10792000FA5B02000000000000022000FA5B020087
:107930000000000000022000FA5B020000000000CE
:1079400000022000FA5B020000000000000220009C
:10795000FA5B02000000000000022000FA5B020057
:107960000000000000022000FA5B0200000000009E
:1079700000022000FA5B02000000000044492000E1
:10798000600420007C5C020000000000F30F200077
:1079900003006200FA5B0200000000004822DE00E3
:1079A00003006200FA5B02000000000020042000D7
:1079B0007C5C02000000000000022000FA5B020074
:1079C0000000000000022000FA5B0200000000003E
:1079D00050052000FA5B02000000000000052000B6
:1079E000FA5B02000000000000022000FA5B0200C7
:1079F0000000000000022000FA5B0200000000000E
:107A000000022000FA5B02000000000000022000DB
:107A1000FA5B02000000000000022000FA5B020096
:107A20000000000000022000FA5B020000000000DD
:107A300000022000FA5B02000000000000022000AB
:107A4000FA5B02000000000040042000FA5B020024
:107A500000000000F0042000FA5B020000000000BB
:107A600070052000FA5B020000000000E004200026
:107A7000FA5B02000000000000022000FA5B020036
:107A80000000000000022000FA5B0200000000007D
:107A900000022000FA5B020000000000000220004B
:107AA000FA5B02000000000000022000FA5B020006
:107AB0000000000000022000FA5B0200000000004D
:107AC00030052000FA5B02000000000040052000A5
:107AD000FA5B020000000000F0042000FA5B0200E4
:107AE0000000000020052000FA5B020000000000FA
:107AF00050042000FA5B020000000000D0012000CA
:107B0000108188008E0B04000000000084482000D3
:107B1000600420007C5C020000000000F30F2000E5
:107B200003006200FA5B0200000000004822DE0051
:107B300003006200FA5B0200000000002004200045
:107B40007C5C02000000000000022000FA5B0200E2
:107B50000000000000022000FA5B020000000000AC
:107B600000022000FA5B0200000000002004200058
:107B7000FA5B02000000000010042000FA5B020023
:107B80000000000030042000FA5B0200000000004A
:107B9000B0042000FA5B0200000000000002200098
:107BA000FA5B02000000000000022000FA5B020005
:107BB0000000000044492000600420007C5C0200BA
:107BC00000000000F30F200003006200FA5B0200D7
:107BD000000000004822DE0003006200FA5B0200A1
:107BE00000000000200420007C5C02000000000077
:107BF00060042000FA5B02000000000090042000F6
:107C0000FA5B02000000000020052000FA5B020081
:107C10000000000030052000FA5B020000000000B8
:107C200040052000FA5B0200000000000002200076
:107C3000FA5B02000000000030052000FA5B020041
:107C40000000000050042000FA5B02000000000069
:107C5000C0042000FA5B0200000000005004200075
:107C6000FA5B02000000000030042000FA5B020012
:107C70000000000040052000FA5B02000000000048
:107C800000022000FA5B02000000000090042000C7
:107C9000FA5B02000000000040052000FA5B0200D1
:107CA0000000000050042000FA5B02000000000009
:107CB000D0042000FA5B0200000000000002200057
:107CC000FA5B02000000000040052000FA5B0200A1
:107CD00000000000F0042000FA5B02000000000039
:107CE00000022000FA5B02000000000010042000E7
:107CF000FA5B02000000000040042000FA5B020072
:107D000000000000A0042000FA5B02000000000058
:107D100050052000FA5B0200000000003005200042
:107D2000FA5B02000000000040052000FA5B020040
:107D30000000000000712200E08288001001200095
:107D4000108188008E0B0400000000008448200091
:107D5000600420007C5C020000000000F30F2000A3
:107D600003006200FA5B0200000000004822DE000F
:107D700003006200FA5B0200000000002004200003
:107D80007C5C02000000000000022000FA5B0200A0
:107D90000000000000022000FA5B0200000000006A
:107DA00000022000FA5B0200000000000002200038
:107DB000FA5B02000000000000022000FA5B0200F3
:107DC0000000000000022000FA5B0200000000003A
:107DD00000022000FA5B0200000000000002200008
:107DE000FA5B02000000000000022000FA5B0200C3
:107DF0000000000044492000600420007C5C020078
:107E000000000000F30F200003006200FA5B020094
:107E1000000000004822DE0003006200FA5B02005E
:107E200000000000200420007C5C02000000000034
:107E300000022000FA5B02000000000000022000A7
:107E4000FA5B02000000000050052000FA5B02000F
:107E50000000000000052000FA5B020000000000A6
:107E600000022000FA5B0200000000000002200077
:107E7000FA5B02000000000000022000FA5B020032
:107E80000000000000022000FA5B02000000000079
:107E900000022000FA5B0200000000000002200047
:107EA000FA5B02000000000000022000FA5B020002
:107EB0000000000000022000FA5B02000000000049
:107EC00040042000FA5B020000000000F0042000E3
:107ED000FA5B02000000000070052000FA5B02005F
:107EE00000000000E0042000FA5B02000000000037
:107EF00000022000FA5B02000000000000022000E7
:107F0000FA5B02000000000000022000FA5B0200A1
:107F10000000000000022000FA5B020000000000E8
:107F200000022000FA5B02000000000000022000B6
:107F3000FA5B02000000000030052000FA5B02003E
:107F40000000000040052000FA5B02000000000075
:107F5000F0042000FA5B0200000000002005200071
:107F6000FA5B02000000000050042000FA5B0200EF
:107F700000000000F0012000108188008E0B04003A
:107F80000000000070838000908288003043200051
:107F9000B082880000002000C0828800821F02009A
:107FA00000000000908280007083880084482000D8
:107FB000600420007C5C020000000000F30F200041
:107FC00003006200FA5B0200000000004822DE00AD
:107FD00003006200FA5B02000000000020042000A1
:107FE0007C5C02000000000000022000FA5B02003E
:107FF0000000000000022000FA5B02000000000008
:1080000000022000FA5B02000000000020042000B3
:10801000FA5B02000000000010042000FA5B02007E
:108020000000000030042000FA5B020000000000A5
:10803000B0042000FA5B02000000000000022000F3
:10804000FA5B02000000000000022000FA5B020060
:108050000000000044492000600420007C5C020015
:1080600000000000F30F200003006200FA5B020032
:10807000000000004822DE0003006200FA5B0200FC
:1080800000000000200420007C5C020000000000D2
:1080900060042000FA5B0200000000009004200051
:1080A000FA5B02000000000020052000FA5B0200DD
:1080B0000000000030052000FA5B02000000000014
:1080C00040052000FA5B02000000000000022000D2
:1080D000FA5B02000000000030052000FA5B02009D
:1080E0000000000050042000FA5B020000000000C5
:1080F000C0042000FA5B02000000000050042000D1
:10810000FA5B02000000000030042000FA5B02006D
:108110000000000040052000FA5B020000000000A3
:1081200000022000FA5B0200000000009004200022
:10813000FA5B02000000000040052000FA5B02002C
:108140000000000050042000FA5B02000000000064
:10815000D0042000FA5B02000000000000022000B2
:10816000FA5B02000000000040052000FA5B0200FC
:1081700000000000F0042000FA5B02000000000094
:1081800000022000FA5B0200000000001004200042
:10819000FA5B02000000000040042000FA5B0200CD
:1081A00000000000A0042000FA5B020000000000B4
:1081B00050052000FA5B020000000000300520009E
:1081C000FA5B02000000000040052000FA5B02009C
:1081D0000000000000712200E082880010012000F1
:1081E000108188008E0B040000000000545D020026
:1081F00000000000B4072000600420007C5C020046
:1082000000000000F30F200003006200FA5B020090
:10821000000000004822DE0003006200FA5B02005A
:1082200000000000200420007C5C02000000000030
:1082300030042000FA5B0200000000000002200071
:10824000FA5B02000000000010042000FA5B02004C
:108250000000000000022000FA5B020000000000A5
:10826000C0042000FA5B02000000000000022000B1
:10827000FA5B02000000000090042000FA5B02009C
:108280000000000000022000FA5B02000000000075
:1082900020042000FA5B0200000000000002200021
:1082A000FA5B02000000000020052000FA5B0200DB
:1082B0000000000000022000FA5B02000000000045
:1082C00010042000FA5B0200000000000002200001
:1082D000FA5B02000000000040052000FA5B02008B
:1082E0000000000000022000FA5B02000000000015
:1082F00090042000FA5B0200000000000002200051
:10830000FA5B020000000000F0042000FA5B0200AB
:108310000000000000022000FA5B020000000000E4
:10832000E0042000FA5B020000000000340A200094
:10833000600420007C5C020000000000F30F2000BD
:1083400003006200FA5B0200000000004822DE0029
:1083500003006200FA5B020000000000200420001D
:108360007C5C020000000000D0022000FA5B0200EA
:1083700000000000D0022000FA5B020000000000B4
:10838000D0022000FA5B020000000000D0022000B2
:10839000FA5B020000000000D0022000FA5B02003D
:1083A00000000000D0022000FA5B02000000000084
:1083B000D0022000FA5B020000000000D002200082
:1083C000FA5B020000000000D0022000FA5B02000D
:1083D00000000000D0022000FA5B02000000000054
:1083E000D0022000FA5B020000000000D002200052
:1083F000FA5B020000000000D0022000FA5B0200DD
:1084000000000000D0022000FA5B02000000000023
:10841000D0022000FA5B020000000000D002200021
:10842000FA5B020000000000D0022000FA5B0200AC
:1084300000000000D0022000FA5B020000000000F3
:10844000D0022000FA5B020000000000D0022000F1
:10845000FA5B020000000000D0022000FA5B02007C
:1084600000000000D4242000600420007C5C020096
:1084700000000000F30F200003006200FA5B02001E
:10848000000000004822DE0003006200FA5B0200E8
:1084900000000000200420007C5C020000000000BE
:1084A00030052000FA5B02000000000000052000FB
:1084B000FA5B02000000000050042000FA5B02009A
:1084C0000000000050042000FA5B020000000000E1
:1084D00040042000FA5B0200000000002427200076
:1084E000600420007C5C020000000000F30F20000C
:1084F00003006200FA5B0200000000004822DE0078
:1085000003006200FA5B020000000000200420006B
:108510007C5C020000000000D0062000FA5B020034
:1085200000000000D0062000FA5B020000000000FE
:10853000F0022000FA5B02000000000000072000AB
:10854000FA5B02000000000050072000FA5B020006
:1085500000000000C0062000FA5B020000000000DE
:1085600030072000FA5B02000000000050062000E7
:10857000FA5B02000000000000022000FA5B02002B
:1085800000000000E08080008081880056620200C8
:108590000000000050828000010320000100400024
:1085A000FA5B0200000000006082800001032000EE
:1085B00001004000FA5B02000000000070828000B1
:1085C0000103200001004000FA5B020000000000EF
:1085D000808280000103200001004000FA5B02005D
:1085E0000000000084482000600420007C5C020041
:1085F00000000000F30F200003006200FA5B02009D
:10860000000000004822DE0003006200FA5B020066
:1086100000000000200420007C5C0200000000003C
:10862000D0042000FA5B02000000000010042000CB
:10863000FA5B02000000000090042000FA5B0200D8
:1086400000000000E0042000FA5B020000000000CF
:1086500000022000FA5B020000000000D0042000AD
:10866000FA5B02000000000050042000FA5B0200E8
:1086700000000000E0042000FA5B0200000000009F
:1086800050052000FA5B0200000000004449200071
:10869000600420007C5C020000000000F30F20005A
:1086A00003006200FA5B0200000000004822DE00C6
:1086B00003006200FA5B02000000000020042000BA
:1086C0007C5C02000000000060042000FA5B0200F5
:1086D0000000000090042000FA5B0200000000008F
:1086E00020052000FA5B0200000000003005200099
:1086F000FA5B02000000000040052000FA5B020067
:108700000000000000022000FA5B020000000000F0
:1087100030052000FA5B0200000000005004200039
:10872000FA5B020000000000C0042000FA5B0200B7
:108730000000000050042000FA5B0200000000006E
:1087400030042000FA5B0200000000004005200019
:10875000FA5B02000000000000022000FA5B020049
:108760000000000090042000FA5B020000000000FE
:1087700040052000FA5B02000000000050042000C9
:10878000FA5B020000000000D0042000FA5B020047
:108790000000000000022000FA5B02000000000060
:1087A00040052000FA5B020000000000F0042000F9
:1087B000FA5B02000000000000022000FA5B0200E9
:1087C0000000000010042000FA5B0200000000001E
:1087D00040042000FA5B020000000000A00420001A
:1087E000FA5B02000000000050052000FA5B020066
:1087F0000000000030052000FA5B020000000000CD
:1088000040052000FA5B0200000000000071220019
:10881000E0828800D0002000108188008E0B0400C8
:1088200000000000A0C680003100200001005000C0
:108830004220AE002E44040000000000722102001D
:108840000000000042730200000000002000200031
:10885000108188004644040000000000A0C680008B
:1088600081002000010050004220AE004644040078
:108870000000000072210200000000000002200041
:108880001081880046440400000000008E0B0400A4
:108890000000000084482000600420007C5C02008E
:1088A00000000000F30F200003006200FA5B0200EA
:1088B000000000004822DE0003006200FA5B0200B4
:1088C00000000000200420007C5C0200000000008A
:1088D00000022000FA5B02000000000000022000FD
:1088E000FA5B02000000000000022000FA5B0200B8
:1088F0000000000000022000FA5B020000000000FF
:1089000000022000FA5B02000000000000022000CC
:10891000FA5B02000000000000022000FA5B020087
:108920000000000000022000FA5B020000000000CE
:1089300000022000FA5B0200000000004449200011
:10894000600420007C5C020000000000F30F2000A7
:1089500003006200FA5B0200000000004822DE0013
:1089600003006200FA5B0200000000002004200007
:108970007C5C02000000000000022000FA5B0200A4
:108980000000000000022000FA5B0200000000006E
:1089900050052000FA5B02000000000000052000E6
:1089A000FA5B02000000000000022000FA5B0200F7
:1089B0000000000000022000FA5B0200000000003E
:1089C00000022000FA5B020000000000000220000C
:1089D000FA5B02000000000000022000FA5B0200C7
:1089E0000000000000022000FA5B0200000000000E
:1089F00000022000FA5B02000000000000022000DC
:108A0000FA5B02000000000040042000FA5B020054
:108A100000000000F0042000FA5B020000000000EB
:108A200070052000FA5B020000000000E004200056
:108A3000FA5B02000000000000022000FA5B020066
:108A40000000000000022000FA5B020000000000AD
:108A500000022000FA5B020000000000000220007B
:108A6000FA5B02000000000000022000FA5B020036
:108A70000000000000022000FA5B0200000000007D
:108A800030052000FA5B02000000000040052000D5
:108A9000FA5B020000000000F0042000FA5B020014
:108AA0000000000020052000FA5B0200000000002A
:108AB00050042000FA5B02000000000010022000B9
:108AC000108188008E0B040000000000E080800010
:108AD00090828800B0272000B0828800000020002B
:108AE000C0828800821F0200000000009082800087
:108AF000E080880084482000600420007C5C020044
:108B000000000000F30F200003006200FA5B020087
:108B1000000000004822DE0003006200FA5B020051
:108B200000000000200420007C5C02000000000027
:108B3000D0042000FA5B02000000000010042000B6
:108B4000FA5B02000000000090042000FA5B0200C3
:108B500000000000E0042000FA5B020000000000BA
:108B600000022000FA5B020000000000D004200098
:108B7000FA5B02000000000050042000FA5B0200D3
:108B800000000000E0042000FA5B0200000000008A
:108B900050052000FA5B020000000000444920005C
:108BA000600420007C5C020000000000F30F200045
:108BB00003006200FA5B0200000000004822DE00B1
:108BC00003006200FA5B02000000000020042000A5
:108BD0007C5C02000000000060042000FA5B0200E0
:108BE0000000000090042000FA5B0200000000007A
:108BF00020052000FA5B0200000000003005200084
:108C0000FA5B02000000000040052000FA5B020051
:108C10000000000000022000FA5B020000000000DB
:108C200030052000FA5B0200000000005004200024
:108C3000FA5B020000000000C0042000FA5B0200A2
:108C40000000000050042000FA5B02000000000059
:108C500030042000FA5B0200000000004005200004
:108C6000FA5B02000000000000022000FA5B020034
:108C70000000000090042000FA5B020000000000E9
:108C800040052000FA5B02000000000050042000B4
:108C9000FA5B020000000000D0042000FA5B020032
:108CA0000000000000022000FA5B0200000000004B
:108CB00040052000FA5B020000000000F0042000E4
:108CC000FA5B02000000000000022000FA5B0200D4
:108CD0000000000010042000FA5B02000000000009
:108CE00040042000FA5B020000000000A004200005
:108CF000FA5B02000000000050052000FA5B020051
:108D00000000000030052000FA5B020000000000B7
:108D100040052000FA5B0200000000000071220004
:108D2000E0828800D0002000108188008E0B0400B3
:108D300000000000545D020000000000E41120006B
:108D4000600420007C5C020000000000F30F2000A3
:108D500003006200FA5B0200000000004822DE000F
:108D600003006200FA5B0200000000002004200003
:108D70007C5C02000000000000052000FA5B02009D
:108D80000000000000022000FA5B0200000000006A
:108D9000F0042000FA5B0200000000000002200046
:108DA000FA5B02000000000070052000FA5B020080
:108DB0000000000000022000FA5B0200000000003A
:108DC00050042000FA5B02000000000000022000B6
:108DD000FA5B02000000000020052000FA5B0200A0
:108DE0000000000000022000FA5B0200000000000A
:108DF00000022000FA5B02000000000000022000D8
:108E0000FA5B020000000000F0042000FA5B0200A0
:108E10000000000000022000FA5B020000000000D9
:108E200060042000FA5B0200000000000002200045
:108E3000FA5B02000000000060042000FA5B020000
:108E40000000000064142000600420007C5C02002C
:108E500000000000F30F200003006200FA5B020034
:108E6000000000004822DE0003006200FA5B0200FE
:108E700000000000200420007C5C020000000000D4
:108E8000D0022000FA5B020000000000D0022000A7
:108E9000FA5B020000000000D0022000FA5B020032
:108EA00000000000D0022000FA5B02000000000079
:108EB000D0022000FA5B020000000000D002200077
:108EC000FA5B020000000000D0022000FA5B020002
:108ED00000000000D0022000FA5B02000000000049
:108EE000D0022000FA5B020000000000D002200047
:108EF000FA5B020000000000D0022000FA5B0200D2
:108F000000000000D0022000FA5B02000000000018
:108F1000D0022000FA5B020000000000D002200016
:108F2000FA5B020000000000D0022000FA5B0200A1
:108F300000000000D0022000FA5B020000000000E8
:108F4000D0022000FA5B0200000000000423200091
:108F5000600420007C5C020000000000F30F200091
:108F600003006200FA5B0200000000004822DE00FD
:108F700003006200FA5B02000000000020042000F1
:108F80007C5C02000000000000052000FA5B02008B
:108F900000000000F0042000FA5B02000000000066
:108FA00070052000FA5B0200000000005004200061
:108FB000FA5B02000000000020052000FA5B0200BE
:108FC0000000000000022000FA5B02000000000028
:108FD000F0042000FA5B02000000000060042000A2
:108FE000FA5B02000000000060042000FA5B02004F
:108FF0000000000014252000600420007C5C0200BA
:1090000000000000F30F200003006200FA5B020082
:10901000000000004822DE0003006200FA5B02004C
:1090200000000000200420007C5C02000000000022
:1090300030042000FA5B0200000000001004200051
:10904000FA5B020000000000E0042000FA5B02006E
:109050000000000030042000FA5B02000000000065
:1090600050042000FA5B020000000000C004200051
:10907000FA5B02000000000064252000600420006C
:109080007C5C020000000000F30F2000030062007F
:10909000FA5B0200000000004822DE0003006200CC
:1090A000FA5B02000000000080382100E0828800A6
:1090B0002230EC008E0B040000000000A0C68000EF
:1090C00011002000010050004220AE007048040052
:1090D0000000000075AEA900A81B040000000000FD
:1090E000A0C6800081002000010050004220AE0098
:1090F0008848040000000000722102000000000007
:109100002000200010818800A81B0400000000003F
:109110005C10E2004220AE0098480400000000000D
:109120002000200010818800984804000000000002
:109130008E0B040000000000545D020000000000DF
:10914000D4112000600420007C5C020000000000BC
:10915000F30F200003006200FA5B02000000000031
:109160004822DE0003006200FA5B020000000000FB
:10917000200420007C5C020000000000400420006D
:10918000FA5B02000000000000022000FA5B02000F
:109190000000000010042000FA5B02000000000044
:1091A00000022000FA5B02000000000040052000E1
:1091B000FA5B02000000000000022000FA5B0200DF
:1091C0000000000010042000FA5B02000000000014
:1091D00000022000FA5B02000000000000022000F4
:1091E000FA5B02000000000000022000FA5B0200AF
:1091F00000000000D0042000FA5B02000000000024
:1092000000022000FA5B02000000000010042000B1
:10921000FA5B02000000000000022000FA5B02007E
:1092200000000000E0042000FA5B020000000000E3
:1092300000022000FA5B0200000000001004200081
:10924000FA5B02000000000000022000FA5B02004E
:109250000000000070042000FA5B02000000000023
:1092600000022000FA5B0200000000005004200011
:10927000FA5B02000000000000022000FA5B02001E
:1092800000000000D0042000FA5B02000000000093
:1092900000022000FA5B02000000000050042000E1
:1092A000FA5B02000000000000022000FA5B0200EE
:1092B00000000000E0042000FA5B02000000000053
:1092C00000022000FA5B02000000000040052000C0
:1092D000FA5B02000000000054142000600420002B
:1092E0007C5C020000000000F30F2000030062001D
:1092F000FA5B0200000000004822DE00030062006A
:10930000FA5B020000000000200420007C5C0200E8
:1093100000000000D0022000FA5B02000000000004
:10932000D0022000FA5B020000000000D002200002
:10933000FA5B020000000000D0022000FA5B02008D
:1093400000000000D0022000FA5B020000000000D4
:10935000D0022000FA5B020000000000D0022000D2
:10936000FA5B020000000000D0022000FA5B02005D
:1093700000000000D0022000FA5B020000000000A4
:10938000D0022000FA5B020000000000D0022000A2
:10939000FA5B020000000000D0022000FA5B02002D
:1093A00000000000D0022000FA5B02000000000074
:1093B000D0022000FA5B020000000000D002200072
:1093C000FA5B020000000000D0022000FA5B0200FD
:1093D00000000000D0022000FA5B02000000000044
:1093E000D0022000FA5B020000000000D002200042
:1093F000FA5B020000000000D0022000FA5B0200CD
:1094000000000000D0022000FA5B02000000000013
:10941000D0022000FA5B020000000000D002200011
:10942000FA5B020000000000D0022000FA5B02009C
:1094300000000000D0022000FA5B020000000000E3
:10944000D0022000FA5B020000000000D0022000E1
:10945000FA5B020000000000D0022000FA5B02006C
:1094600000000000D0022000FA5B020000000000B3
:1094700004232000600420007C5C02000000000047
:10948000F30F200003006200FA5B020000000000FE
:109490004822DE0003006200FA5B020000000000C8
:1094A000200420007C5C020000000000300420004A
:1094B000FA5B020000000000C0042000FA5B02001A
:1094C0000000000050042000FA5B020000000000D1
:1094D00010042000FA5B02000000000020052000BC
:1094E000FA5B020000000000342520006004200028
:1094F0007C5C020000000000F30F2000030062000B
:10950000FA5B0200000000004822DE000300620057
:10951000FA5B020000000000200420007C5C0200D6
:109520000000000030052000FA5B0200000000008F
:1095300050042000FA5B020000000000E00420005C
:10954000FA5B02000000000040042000FA5B020009
:1095500000000000B4402000600420007C5C020099
:1095600000000000F30F200003006200FA5B02001D
:10957000000000004822DE0003006200FA5B0200E7
:1095800000000000200420007C5C020000000000BD
:1095900040042000FA5B020000000000500520009B
:1095A000FA5B020000000000D0042000FA5B020019
:1095B0000000000000052000FA5B0200000000002F
:1095C00084482000600420007C5C02000000000051
:1095D000F30F200003006200FA5B020000000000AD
:1095E0004822DE0003006200FA5B02000000000077
:1095F000200420007C5C0200000000002004200009
:10960000FA5B02000000000010042000FA5B020078
:109610000000000030042000FA5B0200000000009F
:10962000B0042000FA5B0200000000008038210036
:10963000E08288002230EC008E0B04000000000065
:10964000A0C6800031002000010050004220AE0082
:10965000384B0400000000007221020000000000EE
:109660002000200010818800464D0400000000000A
:10967000A0C6800011002000010050004220AE0072
:109680005C4B0400000000000000200010948800E3
:109690000000200020948800E0C68000D0C688002A
:1096A00000002000C0C6880080382100E0828800C9
:1096B000464D040000000000A0C68000810020008C
:1096C000010050004220AE00464C040000000000A3
:1096D00072210200000000005004200064680200B3
:1096E0000000000020042000646802000000000068
:1096F00000032000646802000000000080032000D6
:109700006468020000000000C004200064680200D9
:1097100000000000F0062000646802000000000065
:10972000700620006468020000000000E0032000D2
:109730006468020000000000F0938000309488000C
:10974000009480004094880000002000F09388007E
:10975000000020000094880015EEA90015CEA90095
:1097600015AEA8000000000000000000000000008E
:1097700000000000000000000000000000000000E9
:10978000156EA900000000000000000000000000AD
:1097900000000000000000000000000000000000C9
:1097A000800E2000E25902000000000000002000AE
:1097B000E25902000000000000002000E25902000F
:1097C0000000000000002000E2590200000000003C
:1097D00000002000E259020000000000000020000C
:1097E000E25902000000000000002000E2590200DF
:1097F0000000000000002000E2590200000000000C
:10980000365A020000000000F6740200000000005A
:10981000100020007E32B4000000200080B2B400AE
:10982000F0938000019480001294800023948000C3
:1098300000005100818059004200AF00004C04003C
:109840000000000030948000F09388004094800075
:109850000094880015EEA90015CEA90015AEA90048
:1098600000000000000000000000000000000000F8
:10987000000000000000000000000000803821000F
:10988000E0828800464D040000000000A0C6800071
:1098900071002000010050004220AE00364D04004F
:1098A00000000000722102000000000050042000AF
:1098B00064680200000000002004200064680200C8
:1098C00000000000000320006468020000000000A7
:1098D00080032000646802000000000040042000B3
:1098E0006468020000000000500720006468020065
:1098F00000000000D00620006468020000000000A4
:10990000000720006468020000000000E00320005F
:109910006468020000000000F0938000309488002A
:10992000009480004094880000002000F09388009C
:10993000000020000094880015EEA90015CEA900B3
:1099400015AEA800000000000000000000000000AC
:109950000000000000000000000000000000000007
:10996000156EA900000000000000000000000000CB
:1099700000000000000000000000000000000000E7
:10998000800E2000E25902000000000000002000CC
:10999000E25902000000000000002000E25902002D
:1099A0000000000000002000E2590200000000005A
:1099B00000002000E259020000000000000020002A
:1099C000E25902000000000000002000E2590200FD
:1099D0000000000000002000E2590200000000002A
:1099E000365A020000000000F67402000000000079
:1099F000100020007E32B4000000200080B2B400CD
:109A0000F093800001948000F2FF2F00F30020000B
:109A100000005100818059004200AF00F04C04006A
:109A20000000000030948000F09388004094800093
:109A30000094880015EEA90015CEA90015AEA90066
:109A40000000000000000000000000000000000016
:109A5000000000000000000000000000803821002D
:109A6000E0828800464D0400000000005C10E20027
:109A70004220AE00464D04000000000020002000FF
:109A800010818800464D0400000000008E0B040089
:109A900000000000545D0200000000008448200027
:109AA000600420007C5C020000000000F30F200036
:109AB00003006200FA5B0200000000004822DE00A2
:109AC00003006200FA5B0200000000002004200096
:109AD0007C5C020000000000D0042000FA5B020061
:109AE0000000000010042000FA5B020000000000EB
:109AF00090042000FA5B020000000000E004200057
:109B0000FA5B02000000000000022000FA5B020085
:109B100000000000D0042000FA5B020000000000FA
:109B200050042000FA5B020000000000E004200066
:109B3000FA5B02000000000050052000FA5B020002
:109B400000000000B0002000108188008E0B04008F
:109B500000000000A0C6800031002000010050007D
:109B60004220AE00024F04000000000072210200FB
:109B700000000000C629210000002000001B780022
:109B800000402600001B7800E62C21000000200089
:109B9000001B780000402600001B780006302100E2
:109BA00000002000001B780000402600001B780009
:109BB0002633210000002000001B78000040260012
:109BC000001B78004636210000002000001B7800B2
:109BD00000402600001B78006639210000002000AC
:109BE000001B780000402600001B7800863C210006
:109BF00000002000001B780000402600001B7800B9
:109C0000A63F210000002000001B78000040260035
:109C1000001B7800C642210000002000001B7800D5
:109C200000402600001B7800E645210000002000CF
:109C3000001B780000402600001B78000649210028
:109C400000002000001B780000402600001B780068
:109C5000264C210000002000001B78000040260058
:109C6000001B7800464F210000002000001B7800F8
:109C700000402600001B78006652210000002000F2
:109C8000001B780000402600001B7800865521004C
:109C900000002000001B780000402600001B780018
:109CA000A658210000002000001B7800004026007C
:109CB000001B7800C65B210000002000001B78001C
:109CC00000402600001B7800E65E21000000200016
:109CD000001B780000402600001B7800066221006F
:109CE00000002000001B780000402600001B7800C8
:109CF0002665210000002000001B7800004026009F
:109D0000001B78004668210000002000001B78003E
:109D100000402600001B7800666B21000000200038
:109D2000001B780000402600001B7800866E210092
:109D300000002000001B780000402600001B780077
:109D4000A671210000002000001B780000402600C2
:109D5000001B7800C674210000002000001B780062
:109D600000402600001B7800E6772100000020005C
:109D7000001B780000402600001B7800067B2100B5
:109D800000002000001B780000402600001B780027
:109D9000267E210000002000001B780000402600E5
:109DA000001B78004681210000002000001B780085
:109DB00000402600001B780066842100000020007F
:109DC000001B780000402600001B780086872100D9
:109DD00000002000001B780000402600001B7800D7
:109DE000A68A210000002000001B78000040260009
:109DF000001B7800200020001081880044580400D7
:109E000000000000030220006A32EC005093800042
:109E100001022000810050004200AE00204F0400EB
:109E2000000000008A5D020000000000B65D020034
:109E3000000000006AB2EF00445804000000000077
:109E4000A628210050938000210320000100B800C3
:109E5000000343006693880016407800F10020005C
:109E60000100600011002000810050004220AE007F
:109E7000644F040000000000509380000000E800E0
:109E800041838000808050004200AE00644F040097
:109E9000000000001660A600EC4F04000000000067
:109EA0001650A70046500400000000001640A00015
:109EB0001650A60054500400000000001640A100F7
:109EC00046500400000000006693800081002000DE
:109ED00006834000160278000000200000024200C5
:109EE000600420007C5C020000000000F30F2000F2
:109EF00003006200FA5B0200000000004822DE005E
:109F000003006200FA5B0200000000002004200051
:109F10007C5C0200000000002475020000000000CC
:109F2000669380001660A700C04F04000000000088
:109F300000022000FA5B0200000000000002200086
:109F4000FA5B02000000000000022000FA5B020041
:109F50000000000000022000FA5B02000000000088
:109F600000022000FA5B0200000000000002200056
:109F7000FA5B020000000000E84F0400000000004F
:109F8000C0032000FA5B0200000000004004200033
:109F9000FA5B02000000000050042000FA5B02009F
:109FA0000000000060042000FA5B020000000000D6
:109FB000E0032000FA5B0200000000000002200025
:109FC000FA5B020000000000E84F040000000000FF
:109FD00046500400000000006A12E2004220AF0078
:109FE0000210A800669380008100200006834000D4
:109FF00016027800000020000002420060042000E9
:10A000007C5C020000000000F30F200003006200EF
:10A01000FA5B0200000000004822DE00030062003C
:10A02000FA5B020000000000200420007C5C0200BB
:10A03000000000002475020000000000C0032000A2
:10A04000FA5B02000000000030042000FA5B02000E
:10A0500000000000F0042000FA5B02000000000095
:10A06000D0042000FA5B020000000000E0032000A2
:10A07000FA5B02000000000000022000FA5B020010
:10A080000000000046500400000000008301E900C9
:10A090000300E0004220AE00044F04000000000076
:10A0A00044580400000000000210AF007A51040080
:10A0B000000000006A12E2004220AE004C5504008D
:10A0C0000000000050F627008081880090032000E7
:10A0D0009081880000002000A0818800E08080003E
:10A0E000B08188003830EF003A30EF00AE690200EE
:10A0F00000000000669380005102200006834000AB
:10A1000036407800F10F200001006000B640780072
:10A11000C808DD0002F02F0082806000010070009E
:10A12000B081880036407800F10F20000100600007
:10A13000C0818800669380005102200006834000A1
:10A1400036407800F10F200001006000B640780032
:10A15000C808DD0002F02F0082806000010070005E
:10A16000B1818000810050004220AE007A5004008E
:10A170000000000036407800F10F20000100600070
:10A18000C1818000810050004220AE007A5004005E
:10A19000000000003A30EF00186A020000000000E2
:10A1A00080818000808388006693800041022000C7
:10A1B00006834000364078000030A7007030EF0082
:10A1C000E4442000600420007C5C020000000000E9
:10A1D000F30F200003006200FA5B020000000000A1
:10A1E0004822DE0003006200FA5B0200000000006B
:10A1F000200420007C5C02000000000030052000EC
:10A20000FA5B02000000000000072000FA5B020079
:10A210000000000050062000FA5B02000000000071
:10A2200050062000FA5B02000000000040062000FB
:10A23000FA5B020000000000A0032000FA5B0200AD
:10A240000000000000022000FA5B02000000000095
:10A250008083800080818800566202000000000038
:10A26000408280000103200001004000FA5B0200F0
:10A270000000000050828000010320000100400027
:10A28000FA5B020000000000E0022000FA5B02001E
:10A2900000000000608280000103200001004000F7
:10A2A000FA5B0200000000007082800001032000C1
:10A2B00001004000FA5B020000000000B006200030
:10A2C000FA5B020000000000D0062000FA5B0200EA
:10A2D00000000000F0022000FA5B02000000000015
:10A2E00080062000FA5B0200000000000452040017
:10A2F000000000007030EF006A12E2004220AF0060
:10A300000210A900E4442000600420007C5C0200EC
:10A3100000000000F30F200003006200FA5B02005F
:10A32000000000004822DE0003006200FA5B020029
:10A3300000000000200420007C5C020000000000FF
:10A3400030052000FA5B020000000000000720003A
:10A35000FA5B02000000000050062000FA5B0200D9
:10A360000000000050062000FA5B02000000000020
:10A3700040062000FA5B020000000000A00320005D
:10A38000FA5B02000000000000022000FA5B0200FD
:10A3900000000000C0032000FA5B02000000000083
:10A3A00030042000FA5B020000000000F0042000EE
:10A3B000FA5B020000000000D0042000FA5B0200FB
:10A3C00000000000E0032000FA5B02000000000033
:10A3D00000022000FA5B02000000000000022000E2
:10A3E000FA5B02000000000000022000FA5B02009D
:10A3F0000000000000022000FA5B020000000000E4
:10A400000452040000000000803821007010E200B7
:10A410004220AF00B0C688008016200080818800EE
:10A42000000020009081880000002000A0818800AA
:10A4300000818000B081880000002000C081880079
:10A4400000002000D0818800AE69020000000000FA
:10A45000F0808000B081880000002000C08188006A
:10A4600000002000D0818800AE69020000000000DA
:10A470008081800010828800908180002082880086
:10A48000A08180003082880000A62E008081880094
:10A49000000020009081880000002000A08188003A
:10A4A00080838000B081880000002000C081880087
:10A4B000D0818800AE690200000000008081800029
:10A4C000E081880090818000F0818800A081800078
:10A4D0000082880010838000B08188000000200086
:10A4E000C0818800D0818800AE69020000000000B1
:10A4F00010828000B081880020828000C0818800A6
:10A5000020828000C0818800186A020000000000DC
:10A5100080818000F08288006693800081002000A6
:10A520000683400004002000600420007C5C0200E0
:10A5300000000000F30F200003006200FA5B02003D
:10A54000000000004822DE0003006200FA5B020007
:10A5500000000000200420007C5C020000000000DD
:10A5600000022000FA5B0200000000000002200050
:10A57000FA5B02000000000000022000FA5B02000B
:10A580000000000000022000FA5B02000000000052
:10A5900000022000FA5B0200000000000002200020
:10A5A000FA5B02000000000000022000FA5B0200DB
:10A5B0000000000000022000FA5B02000000000022
:10A5C00000022000FA5B02000000000010838000FF
:10A5D00080818800566202000000000040828000F6
:10A5E0000103200001004000FA5B020000000000AF
:10A5F000508280000103200001004000FA5B02004D
:10A600000000000060828000010320000100400083
:10A61000FA5B02000000000070828000010320004D
:10A6200001004000FA5B0200000000008082800010
:10A630000103200001004000FA5B0200000000005E
:10A64000B0062000FA5B0200000000007006200047
:10A65000FA5B020000000000F0022000FA5B02003A
:10A660000000000080062000FA5B020000000000ED
:10A6700000022000FA5B020000000000000220003F
:10A68000FA5B02000000000000022000FA5B0200FA
:10A690000000000000022000FA5B02000000000041
:10A6A0006693800021012000068340003640780038
:10A6B000F20F20000200600096407800C808DD001C
:10A6C00002F02F008280600001007000808188000D
:10A6D000566202000000000040828000010320005A
:10A6E00001004000FA5B0200000000005082800080
:10A6F0000103200001004000FA5B0200000000009E
:10A70000608280000103200001004000FA5B02002B
:10A710000000000070828000010320000100400062
:10A72000FA5B02000000000080828000010320002C
:10A7300001004000FA5B020000000000D00620008B
:10A74000FA5B020000000000C0062000FA5B020075
:10A7500000000000F0022000FA5B02000000000090
:10A76000D0062000FA5B020000000000000220007A
:10A77000FA5B02000000000000022000FA5B020009
:10A7800000000000A0032000FA5B020000000000AF
:10A7900040052000FA5B02000000000010062000C7
:10A7A000FA5B02000000000020072000FA5B0200B4
:10A7B0000000000070062000FA5B020000000000AC
:10A7C00050062000FA5B0200000000004007200055
:10A7D000FA5B020000000000669380008100200008
:10A7E0000683400004372000600420007C5C0200E7
:10A7F00000000000F30F200003006200FA5B02007B
:10A80000000000004822DE0003006200FA5B020044
:10A8100000000000200420007C5C0200000000001A
:10A8200040052000FA5B0200000000001006200036
:10A83000FA5B02000000000020072000FA5B020023
:10A840000000000070062000FA5B0200000000001B
:10A8500050062000FA5B02000000000040072000C4
:10A86000FA5B020000000000A0032000FA5B020077
:10A870000000000000022000FA5B0200000000005F
:10A8800000022000FA5B020000000000108380003C
:10A890008081880056620200000000004082800033
:10A8A0000103200001004000FA5B020000000000EC
:10A8B000508280000103200001004000FA5B02008A
:10A8C00000000000608280000103200001004000C1
:10A8D000FA5B02000000000070828000010320008B
:10A8E00001004000FA5B020000000000808280004E
:10A8F0000103200001004000FA5B0200000000009C
:10A90000B0062000FA5B0200000000007006200084
:10A91000FA5B020000000000F0022000FA5B020077
:10A920000000000080062000FA5B0200000000002A
:10A9300000022000FA5B020000000000000220007C
:10A94000FA5B02000000000000022000FA5B020037
:10A950000000000000022000FA5B0200000000007E
:10A960006693800021012000068340003640780075
:10A97000F20F20000200600096407800C808DD0059
:10A9800002F02F008280600001007000808188004A
:10A990005662020000000000408280000103200097
:10A9A00001004000FA5B02000000000050828000BD
:10A9B0000103200001004000FA5B020000000000DB
:10A9C000608280000103200001004000FA5B020069
:10A9D00000000000708280000103200001004000A0
:10A9E000FA5B02000000000080828000010320006A
:10A9F00001004000FA5B020000000000D0062000C9
:10AA0000FA5B020000000000C0062000FA5B0200B2
:10AA100000000000F0022000FA5B020000000000CD
:10AA2000D0062000FA5B02000000000000022000B7
:10AA3000FA5B02000000000000022000FA5B020046
:10AA400000000000A0032000FA5B020000000000EC
:10AA500040052000FA5B0200000000001006200004
:10AA6000FA5B02000000000020072000FA5B0200F1
:10AA70000000000070062000FA5B020000000000E9
:10AA800050062000FA5B0200000000004007200092
:10AA9000FA5B020000000000808380006693800063
:10AAA00041012000068340000000E000110020006A
:10AAB0004220AF0001002000014B78006693800027
:10AAC0002001200000034300F0828000F10F2000ED
:10AAD00001006000005B7800F08280004800DE002A
:10AAE00001006000005B7800669380002002200077
:10AAF0000003430016007800F1FF2F008100600082
:10AB00004220AF00B85504000000000000F0A7008C
:10AB1000B85504000000000080818800000020007B
:10AB200090818800A081880010828000B081880018
:10AB300020828000C081880030828000D08188001F
:10AB4000AE69020000000000E0818000B081880052
:10AB5000F0818000C081880000828000D081880060
:10AB6000186A020000000000C05504000000000048
:10AB70000000200080818800C05504000000000013
:10AB80006693800060002000000343008081800005
:10AB9000000B780066938000808180001183800024
:10ABA000010150004200AF00DA550400000000002F
:10ABB0000201EA00A283880010838000808188005F
:10ABC0000000200090818800A0818800A000200063
:10ABD000B081880000002000C0818800D0818800FA
:10ABE000AE6902000000000040062000B08188002D
:10ABF00000002000C0818800D0818800186A02000F
:10AC00000000000080818000A183800001015000CD
:10AC10001670A1004200AE001670A000669380007E
:10AC2000810020000683400016027800000020000A
:10AC300000024200600420007C5C02000000000072
:10AC4000F30F200003006200FA5B02000000000026
:10AC50004822DE0003006200FA5B020000000000F0
:10AC6000200420007C5C020000000000247502002B
:10AC700000000000669380001670A6006A5604006B
:10AC8000000000006130AE006A56040000000000C1
:10AC900000022000FA5B0200000000000002200019
:10ACA000FA5B02000000000000022000FA5B0200D4
:10ACB0000000000000022000FA5B0200000000001B
:10ACC00000022000FA5B020000000000BC560400F5
:10ACD0000000000066938000600020000003430035
:10ACE00016007800808188006593800000032000B2
:10ACF000008042001000A700BC6A020000000000B3
:10AD00005662020000000000408280000103200023
:10AD100001004000FA5B0200000000005082800049
:10AD20000103200001004000FA5B02000000000067
:10AD3000608280000103200001004000FA5B0200F5
:10AD4000000000007082800001032000010040002C
:10AD5000FA5B0200000000008082800001032000F6
:10AD600001004000FA5B0200000000000002200029
:10AD7000FA5B020000000000669380001640A1000C
:10AD8000C43E2000600420007C5C02000000000043
:10AD9000F30F200003006200FA5B020000000000D5
:10ADA0004822DE0003006200FA5B0200000000009F
:10ADB000200420007C5C0200000000004005200010
:10ADC000FA5B02000000000090062000FA5B02001F
:10ADD00000000000D0062000FA5B02000000000026
:10ADE00050062000FA5B020000000000A0032000D3
:10ADF000FA5B02000000000000022000FA5B020083
:10AE000000000000218080004808DE00FA5B02009C
:10AE10000000000020808000FA5B020000000000BB
:10AE2000A0032000FA5B02000000000031808000D7
:10AE30004808DE00FA5B020000000000308080005D
:10AE4000FA5B020000000000A0032000FA5B020091
:10AE500000000000418080004808DE00FA5B02002C
:10AE60000000000040808000FA5B0200000000004B
:10AE700044412000600420007C5C020000000000CF
:10AE8000F30F200003006200FA5B020000000000E4
:10AE90004822DE0003006200FA5B020000000000AE
:10AEA000200420007C5C020000000000C0042000A0
:10AEB000FA5B02000000000010062000FA5B0200AE
:10AEC0000000000040072000FA5B020000000000C4
:10AED000E0022000FA5B020000000000A003200056
:10AEE000FA5B02000000000000022000FA5B020092
:10AEF00000000000518080004808DE00FA5B02007C
:10AF00000000000050808000FA5B0200000000009A
:10AF1000F00D2000FA5B020000000000618080005C
:10AF20004808DE00FA5B020000000000608080003C
:10AF3000FA5B02000000000020022000FA5B020021
:10AF400000000000718080004808DE00FA5B02000B
:10AF50000000000070808000FA5B0200000000002A
:10AF600070022000FA5B0200000000008180800077
:10AF70004808DE00FA5B020000000000C443200025
:10AF8000600420007C5C020000000000F30F200041
:10AF900003006200FA5B0200000000004822DE00AD
:10AFA00003006200FA5B02000000000020042000A1
:10AFB0007C5C020000000000C0042000FA5B02007C
:10AFC00000000000F0062000FA5B02000000000014
:10AFD000E0062000FA5B020000000000700620007E
:10AFE000FA5B020000000000A0032000FA5B0200F0
:10AFF0000000000090808000FA5B0200000000006A
:10B00000A18080004808DE00FA5B0200000000001A
:10B01000A0808000FA5B020000000000F00D20001C
:10B02000FA5B020000000000B18080004808DE00EA
:10B03000FA5B020000000000B0808000FA5B0200B2
:10B040000000000020022000FA5B02000000000067
:10B05000C18080004808DE00FA5B020000000000AA
:10B06000C0808000FA5B0200000000007002200037
:10B07000FA5B020000000000D18080004808DE007A
:10B08000FA5B0200000000008E0B040000000000CC
:10B09000154EA800152EA80015AEA80015CEA900C3
:10B0A00015EEA800000000000000000000000000F5
:10B0B000C05A020000000000000000000000000074
:10B0C00000000000156EA900000000000000000054
:10B0D0000000000000000000000000000000000070
:10B0E00000000000800E2000E25902000000000075
:10B0F00000002000E25902000000000000002000D3
:10B10000E25902000000000000002000E2590200A5
:10B110000000000000002000E259020000000000D2
:10B1200000002000E25902000000000000002000A2
:10B13000E25902000000000000002000E259020075
:10B14000000000000810200009002D00365A0200FF
:10B1500000000000800C78008984E8000804E90001
:10B160000800E0004220AE00A658040000000000E5
:10B17000000000000000000000000000156EA800A4
:10B1800000000000000000000000000000000000BF
:10B19000000000000000000000000000825B0200D0
:10B1A00000000000156EA900000000000000000073
:10B1B000000000000000000000000000000000008F
:10B1C0000000000010082000E2590200000000000A
:10B1D00000002000E25902000000000000002000F2
:10B1E000E25902000000000000002000E2590200C5
:10B1F00000000000156EA800000000000000000024
:10B20000000000000000000000000000000000003E
:10B2100000000000825B020000000000825B020070
:10B2200000000000825B020000000000825B020060
:10B2300000000000156EA9000000000000000000E2
:10B2400000000000000000000000000000000000FE
:10B250000000000040082000E25902000000000049
:10B2600000002000E2590200000000000000200061
:10B27000E25902000000000000002000E259020034
:10B2800000000000081020007000200008004000AE
:10B29000E2590200000000000804E9000800E00094
:10B2A0004220AE004459040000000000156EA800C2
:10B2B000000000000000000000000000000000008E
:10B2C000000000000000000000000000825B02009F
:10B2D00000000000156EA900000000000000000042
:10B2E000000000000000000000000000000000005E
:10B2F0000000000080082000E25902000000000069
:10B3000000002000E25902000000000000002000C0
:10B31000E25902000000000000002000E259020093
:10B3200000000000F0808000E259020000000000F0
:10B3300000818000E25902000000000010838000BC
:10B34000E25902000000000020838000E259020060
:10B350000000000030838000E2590200000000007D
:10B3600040838000E259020000000000508380000A
:10B37000E25902000000000060838000E2590200F0
:10B380000000000070838000E2590200000000000D
:10B39000156EA80000000000000000000000000082
:10B3A000000000000000000000000000000000009D
:10B3B0000000000000000000000000008E0B0400F0
:10B3C00000000000810020000000000000000000DC
:10B3D000000000000000000000000000000000006D
:10B3E00000000000548EA9000000000000000000D2
:10B3F000000000000000000000000000000000004D
:10B40000000000000000D0000080A60035EEA9007A
:10B410000080A70035EEA80000000000000000003A
:10B42000000000000000000000000000000000001C
:10B4300000000000548EA800000000000000000082
:10B4400000000000000000000000000000000000FC
:10B45000000000008100E9000100E0004220AE0091
:10B46000E459040000000000000006000000200075
:10B47000810020000000000000000000000000002B
:10B4800000000000000000000000000000000000BC
:10B49000548EA90000000000000000000000000021
:10B4A000000000000000000000000000000000009C
:10B4B000000000000000000000000000000000008C
:10B4C0000000D00033CEAF000000A00033CEAE00AD
:10B4D0000000A100000000000000000000000000CB
:10B4E000000000000000000000000000000000005C
:10B4F000548EA800000000000000000000000000C2
:10B50000000000000000000000000000000000003B
:10B510008100E9000100E0004220AE003A5A040038
:10B520000000000000000600156EA90000000000E9
:10B53000000000000000000000000000000000000B
:10B540000000000000000000700D2000E259020021
:10B5500000000000365A020000000000156EA8002E
:10B5600000000000000000000000000000000000DB
:10B5700000000000000000000000000000000600C5
:10B58000945A0200000000000070A600C05A040097
:10B59000000000000000A700165B0400000000008F
:10B5A000156EA9000000000000000000000000006F
:10B5B000000000000000000000000000000000008B
:10B5C000D0032000E259020000000000A002200089
:10B5D000E25902000000000000082000E2590200C9
:10B5E00000000000600A2000E25902000000000094
:10B5F000156EA80000000000000000000000000020
:10B60000000000000000000000000000000000003A
:10B61000945A0200000000000070A600085B0400BD
:10B6200000000000085B04000000000000000600AD
:10B63000FFFF3700585B020000000000942EAA00B4
:10B64000585B020000000000942EAA00585B020024
:10B6500000000000942EAA00585B020000000000C9
:10B66000942EAA00585B020000000000942EAA004D
:10B67000585B020000000000942EAA00585B0200F4
:10B6800000000000942EAA00585B02000000000099
:10B69000942EAA00585B020000000000942EAA001D
:10B6A000585B020000000000942EAA000000060073
:10B6B000825B020000000000825B020000000000CC
:10B6C000825B020000000000825B020000000000BC
:10B6D000825B020000000000825B020000000000AC
:10B6E000825B020000000000825B0200000000009C
:10B6F000825B020000000000825B0200000000008C
:10B7000000000600AC5B020000000000AC5B020021
:10B7100000000000AC5B020000000000AC5B020017
:10B7200000000000AC5B020000000000AC5B020007
:10B7300000000000AC5B020000000000AC5B0200F7
:10B7400000000000AC5B020000000000AC5B0200E7
:10B75000000000000000060002022000220888000D
:10B760000021EF0052442000120888000068A90060
:10B7700002022800220888000068AE00BC5B0400BA
:10B780000000000000000600D45B02000000000082
:10B79000C1022000810068004220AE00C45B0400AA
:10B7A00000000000000006002202AE00D45B04008E
:10B7B000000000002682BF00F10F200001006000A1
:10B7C00034A2B7002222AE00EA5B040000000000B1
:10B7D0002222A90000000600004006000000EB0045
:10B7E000000778000C000900002F78000007EB002C
:10B7F00000000600F10F2000810060000500FC0041
:10B8000000F02F00842EB60001007800842EB700CF
:10B810000000000000000000000000000000000028
:10B820000000000000000000000000000000000018
:10B8300000000000348EA90000000000000000009D
:10B8400000000000000000000000000000000000F8
:10B8500000000000000000000000000034AEA9005D
:10B8600000000000000000000000000000000000D8
:10B8700000000000000000000000000000000000C8
:10B880000000000035AEA90000000000000000002C
:10B8900000000000000000000000000000000000A8
:10B8A0000000000000000000000000000000000098
:10B8B0000000000000000000000000000000000088
:10B8C00035AEA800000000000000000000000000ED
:10B8D0000000000000000000000000000000000068
:10B8E000000000000000000034AEA8000A5D020065
:10B8F0000000000000000600F10F20008100600041
:10B900000500FC0000F02F00842EB6000100780036
:10B91000842EB700000000000000000000000000BE
:10B920000000000000000000000000000000000017
:10B930000000000000000000348EA800000000009D
:10B9400000000000000000000000000000000000F7
:10B9500000000000000000000000000000000000E7
:10B9600034AEA9000000000000000000000000004C
:10B9700000000000000000000000000000000000C7
:10B9800000000000000000000000000000000000B7
:10B9900000000000000000000000000000000000A7
:10B9A00035AEA9000000000000000000000000000B
:10B9B0000000000000000000000000000000000087
:10B9C0000000000000000000000000000000000077
:10B9D00000000000000000000000000035AEA800DC
:10B9E0000000000000000000000000000000000057
:10B9F0000000000000000000000000000000000047
:10BA00000000000034AEA8000A5D02000000000043
:10BA10000000060000000000000000000000000020
:10BA20000000000000000000000000000000000016
:10BA30000000000000000000000000000000000006
:10BA400000000000000000000000000000000000F6
:10BA500000000000000000000000000000000000E6
:10BA600000000000000000000000000000000000D6
:10BA700000000000000000000000000000000000C6
:10BA800000000000000000000000000000000000B6
:10BA900000000000000000000000000000000000A6
:10BAA00000000600000006005E5D020000000000CD
:10BAB0008A5D020000000000000006006004200013
:10BAC0007C5C02000000000000002000FA5B020025
:10BAD0000000000000002000FA5B020000000000EF
:10BAE000200420007C5C020000000000084B2000C5
:10BAF00000022000FA5B0200000000000804E900D8
:10BB00000800E0004220AE00785D04000000000064
:10BB100000000600600420007C5C020000000000C1
:10BB200000082000FA5B0200000000005002200024
:10BB3000FA5B020000000000200420007C5C020090
:10BB4000000000000858220000002000FA5B0200FC
:10BB5000000000000804E9000800E0004220AE00F8
:10BB6000A45D040000000000000006008402200024
:10BB700048610200000000008407200048610200C4
:10BB800000000000840C200048610200000000005A
:10BB9000841120004861020000000000841620008B
:10BBA0004861020000000000841B20004861020080
:10BBB0000000000084202000486102000000000016
:10BBC000842520004861020000000000842A200033
:10BBD0004861020000000000842F2000486102003C
:10BBE00000000000843420004861020000000000D2
:10BBF000843920004861020000000000043C20005D
:10BC00004861020000000000044620004861020074
:10BC10000000000004052000600420007C5C02009D
:10BC200000000000F30F200003006200FA5B020036
:10BC3000000000004822DE0003006200FA5B020000
:10BC400000000000200420007C5C020000000000D6
:10BC500020052000FA5B020000000000F006200032
:10BC6000FA5B02000000000070072000FA5B02008F
:10BC70000000000000022000FA5B0200000000004B
:10BC800000022000FA5B020000000000B006200065
:10BC9000FA5B02000000000070062000FA5B020060
:10BCA00000000000F0022000FA5B0200000000002B
:10BCB00080062000FA5B0200000000000002200065
:10BCC000FA5B02000000000020052000FA5B020081
:10BCD00000000000F0062000FA5B020000000000F7
:10BCE00070072000FA5B0200000000000002200044
:10BCF000FA5B02000000000000022000FA5B020074
:10BD000000000000B0062000FA5B02000000000006
:10BD100070062000FA5B020000000000F002200024
:10BD2000FA5B02000000000080062000FA5B0200BF
:10BD30000000000000022000FA5B0200000000008A
:10BD400020052000FA5B020000000000F006200041
:10BD5000FA5B02000000000070072000FA5B02009E
:10BD60000000000000022000FA5B0200000000005A
:10BD700000022000FA5B020000000000B006200074
:10BD8000FA5B02000000000070062000FA5B02006F
:10BD900000000000F0022000FA5B0200000000003A
:10BDA00080062000FA5B0200000000000002200074
:10BDB000FA5B02000000000020052000FA5B020090
:10BDC00000000000F0062000FA5B02000000000006
:10BDD00070072000FA5B0200000000000002200053
:10BDE000FA5B02000000000000022000FA5B020083
:10BDF00000000000B0062000FA5B02000000000016
:10BE000070062000FA5B020000000000F002200033
:10BE1000FA5B02000000000080062000FA5B0200CE
:10BE20000000000000022000FA5B02000000000099
:10BE300004322000600420007C5C0200000000004E
:10BE4000F30F200003006200FA5B02000000000014
:10BE50004822DE0003006200FA5B020000000000DE
:10BE6000200420007C5C020000000000200520006F
:10BE7000FA5B020000000000F0062000FA5B0200FE
:10BE80000000000070072000FA5B020000000000C4
:10BE900000022000FA5B0200000000000002200007
:10BEA000FA5B020000000000B0062000FA5B02000E
:10BEB0000000000070062000FA5B02000000000095
:10BEC000F0022000FA5B0200000000008006200063
:10BED000FA5B02000000000000022000FA5B020092
:10BEE0000000000020052000FA5B020000000000B6
:10BEF000F0062000FA5B020000000000700720003E
:10BF0000FA5B02000000000000022000FA5B020061
:10BF10000000000000022000FA5B020000000000A8
:10BF2000B0062000FA5B020000000000700620004E
:10BF3000FA5B020000000000F0022000FA5B020041
:10BF40000000000080062000FA5B020000000000F4
:10BF500000022000FA5B0200000000002005200023
:10BF6000FA5B020000000000F0062000FA5B02000D
:10BF70000000000070072000FA5B020000000000D3
:10BF800000022000FA5B0200000000000002200016
:10BF9000FA5B020000000000B0062000FA5B02001D
:10BFA0000000000070062000FA5B020000000000A4
:10BFB000F0022000FA5B0200000000008006200072
:10BFC000FA5B02000000000000022000FA5B0200A1
:10BFD0000000000020052000FA5B020000000000C5
:10BFE000F0062000FA5B020000000000700720004D
:10BFF000FA5B02000000000000022000FA5B020071
:10C000000000000000022000FA5B020000000000B7
:10C01000B0062000FA5B020000000000700620005D
:10C02000FA5B020000000000F0022000FA5B020050
:10C030000000000080062000FA5B02000000000003
:10C0400000022000FA5B020000000000B43F200064
:10C050000C610200000000000C6102000000000002
:10C060000C610200000000000C61020000000000F2
:10C0700054422000A6600200000000000C61020093
:10C08000000000000C610200000000000C610200D2
:10C0900000000000D44420005860020000000000AE
:10C0A000E445200058600200000000000000060087
:10C0B000600420007C5C020000000000F30F200000
:10C0C00003006200FA5B0200000000004822DE006C
:10C0D00003006200FA5B0200000000002004200060
:10C0E0007C5C02000000000000022000FA5B0200FD
:10C0F0000000000000000600600420007C5C0200DC
:10C1000000000000F30F200003006200FA5B020051
:10C11000000000004822DE0003006200FA5B02001B
:10C1200000000000200420007C5C020000000000F1
:10C1300000022000FA5B0200000000000002200064
:10C14000FA5B02000000000000000600600420000E
:10C150007C5C020000000000F30F2000030062007E
:10C16000FA5B0200000000004822DE0003006200CB
:10C17000FA5B020000000000200420007C5C02004A
:10C180000000000000022000FA5B02000000000036
:10C1900000022000FA5B0200000000000002200004
:10C1A000FA5B0200000000000000060060042000AE
:10C1B0007C5C020000000000F30F2000030062001E
:10C1C000FA5B0200000000004822DE00030062006B
:10C1D000FA5B020000000000200420007C5C0200EA
:10C1E0000000000000022000FA5B020000000000D6
:10C1F00000022000FA5B02000000000000022000A4
:10C20000FA5B02000000000000022000FA5B02005E
:10C210000000000000000600600420007C5C0200BA
:10C2200000000000F30F200003006200FA5B020030
:10C23000000000004822DE0003006200FA5B0200FA
:10C2400000000000200420007C5C020000000000D0
:10C2500000022000FA5B0200000000000002200043
:10C26000FA5B02000000000000022000FA5B0200FE
:10C270000000000000022000FA5B02000000000045
:10C2800000022000FA5B020000000000000006002F
:10C29000600420007C5C020000000000F30F20001E
:10C2A00003006200FA5B0200000000004822DE008A
:10C2B00003006200FA5B020000000000200420007E
:10C2C0007C5C02000000000000022000FA5B02001B
:10C2D0000000000000022000FA5B020000000000E5
:10C2E00000022000FA5B02000000000000022000B3
:10C2F000FA5B02000000000000022000FA5B02006E
:10C300000000000000022000FA5B020000000000B4
:10C3100000022000FA5B0200000000000002200082
:10C32000FA5B02000000000000022000FA5B02003D
:10C330000000000000022000FA5B02000000000084
:10C3400000022000FA5B0200000000000002200052
:10C35000FA5B02000000000000022000FA5B02000D
:10C360000000000000022000FA5B02000000000054
:10C3700000022000FA5B0200000000000002200022
:10C38000FA5B02000000000000022000FA5B0200DD
:10C390000000000000022000FA5B02000000000024
:10C3A00000022000FA5B02000000000000022000F2
:10C3B000FA5B02000000000000022000FA5B0200AD
:10C3C0000000000000022000FA5B020000000000F4
:10C3D00000022000FA5B02000000000000022000C2
:10C3E000FA5B02000000000000022000FA5B02007D
:10C3F0000000000000022000FA5B020000000000C4
:10C4000000022000FA5B0200000000000002200091
:10C41000FA5B02000000000000022000FA5B02004C
:10C420000000000000022000FA5B02000000000093
:10C4300000022000FA5B0200000000000002200061
:10C44000FA5B02000000000000022000FA5B02001C
:10C450000000000000022000FA5B02000000000063
:10C4600000022000FA5B0200000000000002200031
:10C47000FA5B02000000000000022000FA5B0200EC
:10C480000000000000022000FA5B02000000000033
:10C4900000022000FA5B0200000000000002200001
:10C4A000FA5B020000000000000006004830EF00C8
:10C4B0004A30EF004C30EF004E30EF005030EF00CC
:10C4C0008081800001712200010150004200AE0015
:10C4D0007462040000000000020078004830EC00A4
:10C4E0006462040000000000813E20000101500051
:10C4F0004200AE00866204000000000002007800E6
:10C500004A30EC0076620400000000004106200082
:10C51000010150004200AE009862040000000000DB
:10C52000020078004C30EC0088620400000000003B
:10C53000A1002000010150004200AE00AA620400E8
:10C5400000000000020078004E30EC009A62040007
:10C55000000000008082880000000600A62821005C
:10C560002100200006834000F20F2000020160003D
:10C57000025B7800C800DE00F20F2000028160003C
:10C58000025B7800C62B21002100200006834000BA
:10C59000F20F200002016000025B7800C800DE009C
:10C5A000F20F200002816000025B7800E62E21007D
:10C5B0002100200006834000F20F200002016000ED
:10C5C000025B7800C800DE00F20F200002816000EC
:10C5D000025B780006322100210020000683400023
:10C5E000F20F200002016000025B7800C800DE004C
:10C5F000F20F200002816000025B780026352100E6
:10C600002100200006834000F20F2000020160009C
:10C61000025B7800C800DE00F20F2000028160009B
:10C62000025B78004638210021002000068340008C
:10C63000F20F200002016000025B7800C800DE00FB
:10C64000F20F200002816000025B7800663B21004F
:10C650002100200006834000F20F2000020160004C
:10C66000025B7800C800DE00F20F2000028160004B
:10C67000025B7800863E21002100200006834000F6
:10C68000F20F200002016000025B7800C800DE00AB
:10C69000F20F200002816000025B7800A6412100B9
:10C6A0002100200006834000F20F200002016000FC
:10C6B000025B7800C800DE00F20F200002816000FB
:10C6C000025B7800C6442100210020000683400060
:10C6D000F20F200002016000025B7800C800DE005B
:10C6E000F20F200002816000025B7800E647210023
:10C6F0002100200006834000F20F200002016000AC
:10C70000025B7800C800DE00F20F200002816000AA
:10C71000025B7800064B21002100200006834000C8
:10C72000F20F200002016000025B7800C800DE000A
:10C73000F20F200002816000025B7800264E21008B
:10C740002100200006834000F20F2000020160005B
:10C75000025B7800C800DE00F20F2000028160005A
:10C76000025B780046512100210020000683400032
:10C77000F20F200002016000025B7800C800DE00BA
:10C78000F20F200002816000025B780066542100F5
:10C790002100200006834000F20F2000020160000B
:10C7A000025B7800C800DE00F20F2000028160000A
:10C7B000025B78008657210021002000068340009C
:10C7C000F20F200002016000025B7800C800DE006A
:10C7D000F20F200002816000025B7800A65A21005F
:10C7E0002100200006834000F20F200002016000BB
:10C7F000025B7800C800DE00F20F200002816000BA
:10C80000025B7800C65D2100210020000683400005
:10C81000F20F200002016000025B7800C800DE0019
:10C82000F20F200002816000025B7800E6602100C8
:10C830002100200006834000F20F2000020160006A
:10C84000025B7800C800DE00F20F20000281600069
:10C85000025B78000664210021002000068340006E
:10C86000F20F200002016000025B7800C800DE00C9
:10C87000F20F200002816000025B78002667210031
:10C880002100200006834000F20F2000020160001A
:10C89000025B7800C800DE00F20F20000281600019
:10C8A000025B7800466A21002100200006834000D8
:10C8B000F20F200002016000025B7800C800DE0079
:10C8C000F20F200002816000025B7800666D21009B
:10C8D0002100200006834000F20F200002016000CA
:10C8E000025B7800C800DE00F20F200002816000C9
:10C8F000025B780086702100210020000683400042
:10C90000F20F200002016000025B7800C800DE0028
:10C91000F20F200002816000025B7800A673210004
:10C920002100200006834000F20F20000201600079
:10C93000025B7800C800DE00F20F20000281600078
:10C94000025B7800C67621002100200006834000AB
:10C95000F20F200002016000025B7800C800DE00D8
:10C96000F20F200002816000025B7800E67921006E
:10C970002100200006834000F20F20000201600029
:10C98000025B7800C800DE00F20F20000281600028
:10C99000025B7800067D2100210020000683400014
:10C9A000F20F200002016000025B7800C800DE0088
:10C9B000F20F200002816000025B780026802100D7
:10C9C0002100200006834000F20F200002016000D9
:10C9D000025B7800C800DE00F20F200002816000D8
:10C9E000025B78004683210021002000068340007E
:10C9F000F20F200002016000025B7800C800DE0038
:10CA0000F20F200002816000025B78006686210040
:10CA10002100200006834000F20F20000201600088
:10CA2000025B7800C800DE00F20F20000281600087
:10CA3000025B7800868921002100200006834000E7
:10CA4000F20F200002016000025B7800C800DE00E7
:10CA5000F20F200002816000025B780000000600F7
:10CA60004200F800801F7800811F7800821F780044
:10CA7000B08380000080E800E21321000201500032
:10CA800001003A00A0072100C1838000810050000E
:10CA90004220AF005A650400000000003111800000
:10CAA0000168A90001087800B08388005E65040071
:10CAB00000000000311180000168A9002081800081
:10CAC0000000D000E2032000020060000006010028
:10CAD000F46504000000000004660400000000008B
:10CAE0001A66040000000000306604000000000028
:10CAF00046660400000000005C66040000000000C0
:10CB00007266040000000000886604000000000057
:10CB100092660400000000009E6604000000000011
:10CB2000A866040000000000B466040000000000D5
:10CB3000BE66040000000000CA6604000000000099
:10CB4000DE66040000000000E8660400000000004B
:10CB5000F466040000000000FE660400000000000F
:10CB60000A670400000000001067040000000000D5
:10CB70001A6704000000000026670400000000009F
:10CB80003A67040000000000446704000000000051
:10CB90005A67040000000000646704000000000001
:10CBA0006E670400000000007A67040000000000C7
:10CBB000846704000000000090670400000000008B
:10CBC0009667040000000000A06704000000000059
:10CBD000AC67040000000000C06704000000000013
:10CBE000CA670400000000004202200002816800C1
:10CBF0004220AE0000660400000000002430EC007B
:10CC0000E067040000000000720420000281680058
:10CC10004220AE0014660400000000002430EC0046
:10CC200016660400000000002430EF00E0670400F6
:10CC30000000000002052000028168004220AE00D2
:10CC40002A660400000000002430EC002C6604007A
:10CC5000000000002430EF00E06704000000000046
:10CC600072042000028168004220AE004066040089
:10CC7000000000002430EC004266040000000000C8
:10CC80002430EF00E0670400000000007204200080
:10CC9000028168004220AE005666040000000000D9
:10CCA0002430EC0058660400000000002430EF003F
:10CCB000E067040000000000120420000281680008
:10CCC0004220AE006C660400000000002430EC003E
:10CCD0006E660400000000002430EF00E0670400EE
:10CCE00000000000C2022000028168004220AE0065
:10CCF00082660400000000002430EC00846604001A
:10CD0000000000002430EF00E06704000000000095
:10CD1000C808DD00218088002430EC00E0670400B2
:10CD200000000000208080008100700021808800C9
:10CD30002430EC00E067040000000000C808DD00BB
:10CD4000318088002430EC00E0670400000000001F
:10CD50003080800081007000318088002430EC0039
:10CD6000E067040000000000C808DD004180880082
:10CD70002430EC00E06704000000000040808000E8
:10CD800081007000418088002430EC00E0670400DE
:10CD900000000000C2022000028168004220AE00B4
:10CDA000DA660400000000002430EC00DA660400BB
:10CDB00000000000E067040000000000C808DD007B
:10CDC000518088002430EC00E0670400000000007F
:10CDD0005080800081007000518088002430EC0079
:10CDE000E067040000000000C808DD0061808800E2
:10CDF0002430EC00E0670400000000006080800048
:10CE000081007000618088002430EC00E06704003D
:10CE1000000000002430EC00E06704000000000087
:10CE2000C808DD00718088002430EC00E067040051
:10CE30000000000070808000810070007180880018
:10CE40002430EC00E067040000000000C202200073
:10CE5000028168004220AE00366704000000000036
:10CE60002430EC003667040000000000E067040096
:10CE700000000000C808DD00818088002430EC003C
:10CE8000E067040000000000C20220000281680088
:10CE90004220AE0054670400000000002430EC0083
:10CEA00056670400000000002430EF00E067040033
:10CEB00000000000C808DD00918088002430EC00EC
:10CEC000E067040000000000C808DD00A1808800C1
:10CED0002430EC00E067040000000000A080800027
:10CEE00081007000A18088002430EC00E06704001D
:10CEF00000000000C808DD00B18088002430EC008C
:10CF0000E067040000000000B08080008100700035
:10CF1000B18088002430EC00E067040000000000CD
:10CF20002430EC00E067040000000000C808DD00C9
:10CF3000C18088002430EC00E0670400000000009D
:10CF4000C080800081007000C18088002430EC0027
:10CF5000E067040000000000C202200002816800B7
:10CF60004220AE00BC670400000000002430EC004A
:10CF7000BC67040000000000E0670400000000003F
:10CF8000C808DD00D18088002430EC00E067040090
:10CF900000000000C2022000028168004220AE00B2
:10CFA000DA670400000000002430EF00DC670400B2
:10CFB000000000002430EF00E067040000000000E3
:10CFC0004F017800CF0078004F0078004200F90050
:10CFD000004006004200F800801F7800811F7800A2
:10CFE000821F7800A2680200000000004F01780054
:10CFF000CF0078004F0078004200F90000400600A2
:10D000002222A9000828A900004006003222A90017
:10D010000848A900004006004200F800801F780080
:10D02000811F7800821F780008690200000000005C
:10D030004F017800CF0078004F0078004200F900DF
:10D04000004006004200F800801F7800811F780031
:10D05000821F7800D4680200000000004F017800B1
:10D06000CF0078004F0078004200F9000040060031
:10D070005222A9000A28A90000400600F089800079
:10D08000008A8800018A8000010050004220AE0022
:10D090003E6804000000000000000600319080009F
:10D0A000800878008180E800A226210002815000DB
:10D0B00001003A00A120210031908800158EA900BE
:10D0C0002A68A80000000600118D80008100E80099
:10D0D000522021000281500001003A00611A210013
:10D0E000228D8000028150004220AF007068040051
:10D0F0000000000080487800118D880023E8A80017
:10D1000000000600018A8000F089800001005000C4
:10D110004200A9004220AF00A06804000000000007
:10D120008180E800221A21000281500001003A00AB
:10D130002114210011007800018A88004200A80013
:10D1400000000600218D8000108D8000010050003D
:10D150004220AF00CA680400000000003322AF0084
:10D16000D2680400000000001140780034E2B700EB
:10D170008100E800522021000281500001003A00A5
:10D18000611A2100218D8800956EAA0006690400AD
:10D19000000000003302AE00D2680400000000006E
:10D1A00023E8A90000000600419080003090800034
:10D1B000010050004220AF00FC68040000000000A5
:10D1C0005322AF000669040000000000110078003F
:10D1D000A01288008180E800A22621000281500070
:10D1E00001003A00A120210041908800958EAA00FC
:10D1F00006690400000000005302AE000669040046
:10D20000000000002A68A900158EA8000000060092
:10D210002A68AF003069040000000000F089800037
:10D220000080E800221A21000201500001003A00AB
:10D2300020142100018A8000810050004220AF00AC
:10D240003069040000000000B11280000A48A90003
:10D2500001087800F08988003469040000000000AB
:10D26000B11280000A48A90000000600000000007A
:10D27000000000000000000000000000366904000B
:10D28000000000000000000000000000000000009E
:10D2900000000000426904000000000000000000DF
:10D2A0000000000000000000000000004E690400C3
:10D2B000000000000000000000000000000000006E
:10D2C000000000005A690400000000000000000097
:10D2D000000000000000000000000000666904007B
:10D2E000000000000000000000000000000000003E
:10D2F000000000007269040000000000000000004F
:10D300000000000000000000000000007E69040032
:10D31000000000000000000000000000000000000D
:10D32000000000008A690400000000000000000006
:10D3300000000000000000000000000096690400EA
:10D3400000000000000000000000000000000000DD
:10D35000000000000002040000000000801F7800B0
:10D36000811F7800821F7800831F7800841F780057
:10D37000851F7800861F7800881F7800891F780035
:10D380008A1F78008181800092818000A3818000C3
:10D39000B4818000C5818000D68180000004EB004C
:10D3A0008004EB000005EB00040CB80088818800C5
:10D3B000998188003430EF000414B8000800780028
:10D3C0003230B4000900780034B0B400041CB80056
:10D3D000080078003430B400050CB800080078006C
:10D3E0003230B4000900780034B0B4000514B8003D
:10D3F000080078003430B400060CB800080078004B
:10D400003430B4004F057800CF0478004F04780022
:10D410004F037800CF0278004F027800CF017800E8
:10D420004F017800CF0078004F0078000000060020
:10D43000801F7800811F7800821F7800841F780089
:10D44000851F7800861F7800881F7800891F780064
:10D450008A1F78000003200070818800808180008E
:10D4600091818000A2818000B4818000C58180000C
:10D47000D68180000004EB008004EB000005EB0087
:10D480004200A9002C10AF004200A8000080D2008A
:10D490008180D2000281D2000884D2008984D20027
:10D4A0000A85D2000404540085845C0006055D00F2
:10D4B0002C10A9004200AF002C10A800030031007E
:10D4C0000404440085844C0006054D002E30ED0018
:10D4D0002E10E2004220AE00406A0400000000006E
:10D4E0004200A9002C10AF004200A8000080D2002A
:10D4F0008180D2000281D2008081880091818800E1
:10D50000A28188004F057800CF0478004F0478008E
:10D510004F037800CF0278004F0278004F01780067
:10D52000CF0078004F0078000000060000000600E1
:10D53000801F7800B08180003030B400C08180004E
:10D5400032B0B400D081800034B0B4004F00780015
:10D5500000000600801F7800B08180003030B500E8
:10D56000C081800032B0B500D081800034B0B500F9
:10D570004F00780000000600000006001000A10027
:10D58000B0072000E06A0200000000005093800015
:10D59000E06A020000000000C0022000E06A020011
:10D5A0000000000016007800E06A020000000000A1
:10D5B000D0072000E06A0200000000000000060022
:10D5C000D1C68000800878008180E80062EB2100ED
:10D5D0000281500001003A00E18D2100D1C688008F
:10D5E000D8B8EC0000000600E1C680001100780009
:10D5F0008180E80062EB21000281500001003A00C6
:10D60000E18D2100E1C688000000060005EEA800BB
:10D61000801F7800811F7800821F7800831F7800A8
:10D62000841F7800851F7800861F78006030EC002A
:10D630007230ED007210E2004220AE004E6B04002A
:10D6400000000000803E2000908388004E6B0400A4
:10D650000000000003022000A2282100030078003F
:10D660000000E900210320000100B8000001410092
:10D670001260A600446B04000000000000032000BC
:10D68000000141001200A0008301E9000300E00056
:10D690004220AE002C6B04000000000050C6800049
:10D6A0000000D000E1012000010060000006010040
:10D6B000986B040000000000AA6B0400000000004A
:10D6C000CE6B040000000000F26B040000000000BC
:10D6D0001C6C040000000000986B040000000000B7
:10D6E000986B040000000000986B0400000000002C
:10D6F000986B040000000000986B0400000000001C
:10D70000986B040000000000986B0400000000000B
:10D71000986B040000000000986B040000000000FB
:10D72000986B040000000000986B040000000000EB
:10D73000CC38EF00CEB8EF00850EA800852EA900EA
:10D74000854EA900856EA900CA38EC00DE6C040085
:10D750000000000060C68000838EAE0070C68800A6
:10D760000000E80083AEAE0070C688000000E8004C
:10D7700083CEAE0070C688000000E80060C6880056
:10D78000850EA900852EA800854EA900856EA900EA
:10D79000CA38EC00DE6C04000000000060C68000A7
:10D7A000838EAE0070C688000000E80083AEAE0035
:10D7B00070C688000000E80083CEAE0070C6880006
:10D7C0000000E80060C68800850EA900852EA9002B
:10D7D000854EA800856EA900CA38EC00DE6C0400F6
:10D7E0000000000060C68000838EAE0070C6880016
:10D7F0000000E80083AEAE0070C688000000E800BC
:10D8000083CEAE0070C688000000E80060C68800C5
:10D81000850EA90000000000852EA9000000000070
:10D82000854EA90000000000856EA800CA38EC00F3
:10D83000DE6C04000000000060C68000838EAE0035
:10D8400070C688000000E800CA38EF0070C680008B
:10D8500091C68000010150004220AF003C6C0400E2
:10D860000000000090C68800A000200080C688004C
:10D87000DE6C040000000000D018E2004220AF007F
:10D88000DA6C040000000000D038ED00D018E2008F
:10D890004220AE00DA6C0400000000004200DD000F
:10D8A000C1032000010060000006010020002000EC
:10D8B000A0C68800DA6C0400000000001000200000
:10D8C000A0C68800DA6C0400000000000000200000
:10D8D000A0C68800DA6C04000000000030002000C0
:10D8E000A0C68800DA6C04000000000040002000A0
:10D8F000A0C68800DA6C0400000000005000200080
:10D90000A0C68800DA6C040000000000800020003F
:10D91000A0C68800DA6C040000000000700020003F
:10D92000A0C68800DA6C040000000000600020003F
:10D93000A0C68800DA6C04000000000090002000FF
:10D94000A0C68800DA6C040000000000000000009F
:10D9500000000000000000000000000000000000C7
:10D9600000000000000000000000000000000000B7
:10D9700000000000000000000000000000000000A7
:10D980000000000000000000000000000000000097
:10D990000000000000000000000000000000000087
:10D9A000000000000000000000000000F0FF2F0059
:10D9B000A0C68800DE6C0400000000005C10E200DD
:10D9C0004220AE005C30ED0010818000B1002000EC
:10D9D000010050004220AF00FA6C0400000000007B
:10D9E0000230A90080382100B0C688000A6D04000A
:10D9F00000000000D638ED00D618E2004220AE004C
:10DA00000A6D04000000000080382100B0C68800C4
:10DA10000230A800709380000000D000E1032000D5
:10DA20000100600000060100AC6D04000000000071
:10DA3000B86D040000000000166E04000000000035
:10DA40007C6E040000000000B26E040000000000C4
:10DA5000E86E0400000000003E6F040000000000BB
:10DA6000586F040000000000BC6F040000000000BC
:10DA7000F26F0400000000002A70040000000000A3
:10DA80006C70040000000000C8700400000000007A
:10DA9000E67004000000000038710400000000007F
:10DAA000A271040000000000D87104000000000012
:10DAB0000E72040000000000647204000000000008
:10DAC000AC6D040000000000AC6D0400000000001C
:10DAD000AC6D040000000000AC6D0400000000000C
:10DAE000AC6D040000000000AC6D040000000000FC
:10DAF000AC6D040000000000AC6D040000000000EC
:10DB0000AC6D040000000000AC6D040000000000DB
:10DB1000AC6D040000000000AC6D040000000000CB
:10DB2000AC6D040000000000AC6D040000000000BB
:10DB3000AC6D040000000000AC6D040000000000AB
:10DB4000AC6D040000000000AC6D0400000000009B
:10DB5000AC6D04000000000070B2EF007CB2EF007A
:10DB60001000200070938800827204000000000002
:10DB7000030220007032EC0080938000010220003C
:10DB8000010050004200AE00D26D04000000000011
:10DB900070B2EF00D000200070938800126E040075
:10DBA00000000000A22821008093800021032000B3
:10DBB0000100B800000141009293880012407800F3
:10DBC000F1002000010060004220AF00006E040060
:10DBD000000000001260A600006E040000000000BB
:10DBE0001240A700006E0400000000001250A000C8
:10DBF0002000200070938800126E040000000000D6
:10DC00008301E9000300E0004220AE00BA6D040089
:10DC100000000000D000200070938800126E040005
:10DC20000000000082720400000000009693800053
:10DC30003E68020000000000809380000000E800C1
:10DC400001102000010070004E680200000000007A
:10DC50000002EB00564078004400DE00F100200096
:10DC60000100600080027800040240004E6802005B
:10DC7000000000008502E8001000200004024000BF
:10DC80004E68020000000000000020000402400076
:10DC90004E680200000000009693800020012000E2
:10DCA0000003430036407800040240004E68020042
:10DCB000000000008502E9000500E0004220AE00FF
:10DCC000526E0400000000000480EA00F10F200002
:10DCD000010060004E680200000000009693800082
:10DCE00020032000B093880030002000709388004B
:10DCF0008272040000000000826802000000000040
:10DD00004200AF009C6E0400000000007612E200AA
:10DD10004220AF002A6F0400000000007632ED00C0
:10DD20007612E2004220AE00AE6E04000000000059
:10DD30002A6F04000000000001102000810068002C
:10DD40004220AE002A6F04000000000040002000C6
:10DD500070938800AE6E0400000000003A6F04006B
:10DD60000000000082680200000000004200AF00D6
:10DD7000D26E0400000000007612E2004220AF00E4
:10DD80002A6F0400000000007632ED007612E200F7
:10DD90004220AE00E46E0400000000002A6F040080
:10DDA0000000000011002000810068004220AE0049
:10DDB0002A6F0400000000005000200070938800CB
:10DDC000E46E0400000000003A6F04000000000050
:10DDD00082680200000000004200AF00086F0400EB
:10DDE000000000007612E2004220AF002A6F04001B
:10DDF000000000007632ED007612E2004220AE0014
:10DE0000166F0400000000002A6F040000000000EC
:10DE1000E10F2000810068004220AE002A6F04005C
:10DE2000000000001A6F0400000000003A6F0400B8
:10DE300000000000969380001664A000A00020005F
:10DE4000B093880060002000709388003A6F04004F
:10DE500000000000969380001664A100A00020003E
:10DE6000B0938800C0002000709388003A6F0400CF
:10DE70000000000082720400000000007612E20040
:10DE80004220AF00506F0400000000007632ED0029
:10DE90007612E2004220AE00546F04000000000041
:10DEA000700020007093880082720400000000005F
:10DEB000969380003E68020000000000809380007E
:10DEC0000000E80001102000010070004E68020010
:10DED000000000002630EF0056407800F1002000DE
:10DEE00001006000C0938800010420000100700060
:10DEF0003181800081004000318188004E6802003D
:10DF0000000000007832EC00100020003181800019
:10DF100081004000318188004E680200000000004E
:10DF200000012000318180008100400031818800A3
:10DF30004E68020000000000308180000080EA008E
:10DF4000F10F2000010060004E6802000000000098
:10DF5000969380002002200000034300A6938800CF
:10DF600020032000B0938800800020007093880078
:10DF700082720400000000008268020000000000BD
:10DF80004200AF00DC6F0400000000007612E200E7
:10DF90004220AF00B4700400000000007632ED00B3
:10DFA0007612E2004220AE00EE6F04000000000096
:10DFB000B47004000000000001102000810068001F
:10DFC0004220AE00B4700400000000009000200069
:10DFD00070938800EE6F040000000000C47004001D
:10DFE0000000000082680200000000004200AF0054
:10DFF00012700400000000007612E2004220AF0020
:10E00000B4700400000000007632ED007612E200E9
:10E010004220AE002670040000000000B47004002E
:10E020000000000011002000810068004220AE00C6
:10E03000B470040000000000D0938800A00020000D
:10E04000709388002670040000000000C470040073
:10E050000000000082680200000000004200AF00E3
:10E060004A700400000000007612E2004220AF0077
:10E07000B4700400000000007632ED007612E20079
:10E080004220AE006870040000000000B47004007C
:10E0900000000000A6938000005B7800A693880033
:10E0A000D193800081004000D19388007832ED0048
:10E0B0007812E2004220AE00687004000000000008
:10E0C000B000200070938800687004000000000019
:10E0D000C47004000000000082680200000000001C
:10E0E0004200AF008C700400000000007612E200D5
:10E0F0004220AF00B4700400000000007632ED0052
:10E100007612E2004220AE00A07004000000000081
:10E11000B470040000000000D19380008180EA0008
:10E12000F20F200082806000810050004220AE008B
:10E13000B470040000000000A4700400000000009F
:10E14000C470040000000000969380001664A000D4
:10E15000A0002000B0938800C000200070938800C9
:10E16000C470040000000000969380001664A100B3
:10E17000A0002000B0938800C000200070938800A9
:10E18000C47004000000000082720400000000005F
:10E190007612E2004220AF00DA70040000000000B6
:10E1A0007632ED007612E2004220AE00E27004000A
:10E1B00000000000929380001250A1001000200087
:10E1C00070938800827204000000000003022000A7
:10E1D0007C32EC00E093800001022000010050003E
:10E1E0004200AF007C32EF00A2282100E0938000C3
:10E1F000210320000100B800000141009293880033
:10E2000012407800F1002000010060004220AF00C1
:10E2100022710400000000001260A70022710400B7
:10E22000000000001240A70022710400000000005E
:10E230001250A000E00020007093880034710400A8
:10E24000000000008301E9000300E0004220AE006E
:10E25000E8700400000000001000200070938800A7
:10E26000347104000000000082720400000000000D
:10E27000969380003E68020000000000E09380005A
:10E280000000E80001102000010070004E6802004C
:10E290000000000030002000000278004E680200FC
:10E2A0000000000010002000040240004E68020040
:10E2B0000000000000002000040240004E68020040
:10E2C00000000000F0828000F10F200001006000DB
:10E2D000040240004E68020000000000F08280004E
:10E2E0004800DE00F10F2000010060000402400041
:10E2F0004E680200000000001000200004024000F0
:10E300004E680200000000004006200004024000A9
:10E310004E680200000000000480EA00F10F2000B7
:10E32000010060004E680200000000002003200091
:10E33000B0938800F000200070938800827204007F
:10E340000000000082680200000000004200AF00F0
:10E35000C2710400000000007612E2004220AF000B
:10E3600050720400000000007632ED007612E200E8
:10E370004220AE00D471040000000000507204007E
:10E380000000000001102000810068004220AE0063
:10E39000507204000000000000012000709388000B
:10E3A000D47104000000000060720400000000004E
:10E3B00082680200000000004200AF00F871040013
:10E3C000000000007612E2004220AF00507204000C
:10E3D000000000007632ED007612E2004220AE002E
:10E3E0000A720400000000005072040000000000E7
:10E3F00011002000810068004220AE00507204002D
:10E400000000000010012000709388000A720400D0
:10E41000000000006072040000000000826802003A
:10E42000000000004200AF002E7204000000000057
:10E430007612E2004220AF0050720400000000009B
:10E440007632ED007612E2004220AE003C7204000B
:10E45000000000005072040000000000E10F2000E6
:10E46000810068004220AE005072040000000000ED
:10E470004072040000000000607204000000000010
:10E48000969380001664A000A0002000B09388003E
:10E4900020012000709388006072040000000000DA
:10E4A000969380001664A100A0002000B09388001D
:10E4B00020012000709388006072040000000000BA
:10E4C00082720400000000007612E2004220AF00D9
:10E4D00076720400000000007632ED007612E20051
:10E4E0004220AE007E720400000000009293800083
:10E4F0001250A10010002000709388008272040066
:10E50000000000004F037800CF0278004F0278002F
:10E51000CF0178004F017800CF0078004F007800DD
:10E5200005EEA90000E8A900004006000094800064
:10E530004300DE0000007800156EA9000000000016
:10E5400000000000000000000000000000000000CB
:10E55000000000000000000010082000E259020046
:10E560000000000004948000F30720000300620014
:10E57000E259020000000000F49380004822DE000F
:10E5800003006200E259020000000000F4938000E2
:10E59000F30F200003006200E259020000000000B7
:10E5A000156EA80000000000000000000000000040
:10E5B000000000000000000000000000000000005B
:10E5C000825B020000000000825B0200000000008D
:10E5D000825B020000000000825B0200000000007D
:10E5E00000000600009480004300DE000000780078
:10E5F000156EA900000000000000000000000000EF
:10E60000000000000000000000000000000000000A
:10E6100080082000E25902000000000004948000FD
:10E62000F307200003006200E2590200000000002E
:10E63000F49380004822DE0003006200E2590200E9
:10E6400000000000F4938000F30F2000030062003C
:10E65000E259020000000000156EA8000000000052
:10E6600000000000000000000000000000000000AA
:10E670000000000000000000825B020000000000BB
:10E680000000060015EEA90015CEA90015AEA900E0
:10E69000000000000000000000000000000000007A
:10E6A000000000000000000000000000825B02008B
:10E6B00000000000156EA90000000000000000002E
:10E6C000000000000000000000000000000000004A
:10E6D0000000000010082000E259020000000000C5
:10E6E00000002000E25902000000000000002000AD
:10E6F000E25902000000000000002000E259020080
:10E7000000000000156EA8000000000000000000DE
:10E7100000000000000000000000000000000000F9
:10E7200000000000825B020000000000825B02002B
:10E7300000000000825B020000000000825B02001B
:10E7400000000000156EA90000000000000000009D
:10E7500000000000000000000000000000000000B9
:10E760000000000040082000E25902000000000004
:10E7700000002000E259020000000000000020001C
:10E78000E25902000000000000002000E2590200EF
:10E7900000000000F4808000F30F200003006200FE
:10E7A000E2590200000000004822DE00030062007F
:10E7B000E25902000000000004818000F30F2000F5
:10E7C00003006200E2590200000000004822DE005F
:10E7D00003006200E2590200000000001483800080
:10E7E000F30F200003006200E25902000000000065
:10E7F0004822DE0003006200E2590200000000002F
:10E8000024838000F30F200003006200E25902001D
:10E81000000000004822DE0003006200E25902000E
:10E820000000000034838000F30F2000030062002A
:10E83000E2590200000000004822DE0003006200EE
:10E84000E25902000000000044838000F30F200022
:10E8500003006200E2590200000000004822DE00CE
:10E8600003006200E25902000000000054838000AF
:10E87000F30F200003006200E259020000000000D4
:10E880004822DE0003006200E2590200000000009E
:10E8900064838000F30F200003006200E25902004D
:10E8A000000000004822DE0003006200E25902007E
:10E8B0000000000074838000F30F2000030062005A
:10E8C000E2590200000000004822DE00030062005E
:10E8D000E259020000000000E4808000F30F2000F5
:10E8E00003006200E2590200000000004822DE003E
:10E8F00003006200E259020000000000F49380006F
:10E90000F30F200003006200E25902000000000043
:10E910004822DE0003006200E2590200000000000D
:10E9200004948000F30F200003006200E25902000B
:10E93000000000004822DE0003006200E2590200ED
:10E9400000000000000000000000000000000000C7
:10E95000156EA8000000000000000000000000008C
:10E9600000000000000000000000000000000000A7
:10E97000825B020000000000156EA900000000008C
:10E980000000000000000000000000000000000087
:10E99000000000000000000080082000E259020092
:10E9A0000000000000002000E2590200000000000A
:10E9B00000002000E25902000000000000002000DA
:10E9C000E259020000000000156EA80000000000DF
:10E9D0000000000000000000000000000000000037
:10E9E000000000000000000000000600801F78000A
:10E9F0004400DE00F10020000100600016750200F6
:10EA00000000000064680200000000004F00780071
:10EA1000F1002000010060001675020000000000F7
:10EA2000646802000000000000000600A100200051
:10EA300081005000010320004200AF00710320005C
:10EA40000100400000000600509380000000E80034
:10EA50008081880056620200000000007082800001
:10EA60000103200001004000FA5B020000000000EA
:10EA7000808280000103200001004000FA5B020058
:10EA800000000000A0032000FA5B0200000000006C
:10EA900000022000FA5B02000000000000000600F7
:10EAA0000200000003000000050000000A00000052
:10EAB000001000007E0F0000800000000000000039
:10EAC000FFFFFF00FFFFFF00FFFFFF00FFFFFF0052
:10EAD000FFFFFF00FFFFFF00FFFFFF00FFFFFF0042
:10EAE000FFFFFF00FFFFFF00FFFFFF00FFFFFF0032
:10EAF000FFFFFF00FFFFFF00FFFFFF00FFFFFF0022
:0200000400FFFB
:0200000401F009
:100008000300000083000000250000007F000000BE
:0C00180037000000D500000003000000CD
:04002400FF000000D9
:00000001FF
